:020000041100E9
:10300000002370B5284C0120636101F043FA402091
:103010000223FE21254A207401F0C2FA002833D190
:103020000223FF21224A207C01F0BAFA00282BD18A
:10303000204BA2899A4224D1E3891F4A93420CD1A2
:103040001E4B63611E4B2268002A03D1002B01D066
:1030500023CB23C401F092FA70BD1A4A934201D0E7
:103060000023F0E7184B194A1B68934205D9C02288
:103070000421207C920001F00DFB104B6361144B86
:10308000E1E700232374EBE7CC223820AC21920146
:10309000207401F0FFFA0028F3D10E4B63610E4B50
:1030A000E3810E4BCFE7C0469463FF1FA063FF1F71
:1030B000A263FF1F5959000083050000F54200116B
:1030C00098BA001182150000B863FF1F8713000033
:1030D000A4BA001191430011AAAAFFFF8CBA0011F3
:1030E000F7B5164B0192C318021D002000938823E8
:1030F0005B05D3181B685C1C1AD09CB2402C18D8F6
:103100008D781E0CAC466746CD782D023D43AE420D
:1031100006D1019800280ED110000C70240A4C70C2
:1031200003249BB20733A343D218009B9A42DED3F9
:10313000FEBD4432F9E71000FAE7C046FC0F00007C
:10314000802213B503000324019189B25201073193
:103150009B18A14304305A1A88235B05C3181B68C7
:10316000591C03D190429241104016BD99B240299A
:1031700007D80B000733A343C0189042ECD30020BC
:10318000F3E74430F9E7134B134A1B68126810B594
:10319000FA24934201D81A00F824104BE4021B6869
:1031A0009A4210D813000E4A12689A420ED3013385
:1031B00007D1F823DB029C4203D10A49054808F0F5
:1031C000BFF8200010BDFC24E402ECE7FE24E4027A
:1031D000F7E7C04600C0071100D0071100E0071153
:1031E00000F00711FFFFFF7FF0B59BB015000490C2
:1031F0000391402A00D9A0E006AB59801A80FFF75E
:10320000C2FF0400042816D9002206A9FFF768FFB0
:10321000052810D906AB1B88AB420CD1002D07D076
:10322000514B2A000499C01808F0D2F9002802D1A5
:1032300001201BB0F0BD06AB1D8020000699FFF7F2
:103240007FFF041E7BD1069B0793FFF79CFF802323
:103250005B01C618802307001B039E4201D3F8269A
:10326000F60288235B05F31801931B68013302D033
:10327000019808F0DDF83D49019808F061F83B1D20
:103280000293331D05938822029B52059B181B68ED
:1032900008935A1C3CD044219AB20091402A04D889
:1032A0000320D11D814389B2009103991B0C8B42ED
:1032B00024D0402A22D80122300008A9FFF710FFAD
:1032C000021E1BD1380008A9FFF70AFF04000428DA
:1032D00031D9009A059B9B1880225201B218934263
:1032E00040D288235B05C118009A09A808F070F83D
:1032F0001D4B009A09A9F01808F08AF8009A029B61
:103300009446634402931A4B029AFB189A42BAD32A
:1033100088235B05FC1821680198013908F010F832
:10332000200008F085F8039A07AB5A80300007990F
:10333000FFF706FF0400002C03D1002079E70428E2
:10334000FBD988235B05E018069907F0F9FF0323F2
:10335000EA1C9A4300D16BE7034B0499E01808F08C
:1033600057F865E70424ECE704000011FFFFFF7F36
:10337000F80F0000F7B505001400402A21D80027F7
:1033800001AE71803780FFF7FEFE042816D93A009F
:103390003100FFF7A5FE042810D93688BC420BD0B7
:1033A000BD4209D0221CB44200D9321C064B92B255
:1033B000C118280008F00CF830B2FEBDC04300B2BE
:1033C000FBE703204042F8E70400001137B5042270
:1033D00004000D0001A81649FFF7CCFF02000428E5
:1033E0000BD1019BA34208D3AB4204D0104901A8E2
:1033F0000195FFF7F9FE01203EBD0E4C2368200029
:10340000019308F015F8019920000139019107F0A6
:1034100097FF80235B01E418074B9C42EED1042206
:10342000034901A80195FFF7DFFE0020E4E7C0464D
:103430005555000000C007110000081130B589B0D3
:1034400008F0CEF910226946254808F0F1F8254B1E
:10345000009A9A420ED1019B029A0F2B33D8002179
:1034600001240698013B08D2002900D00292029B59
:10347000013331D10023029325E0551CF2D1020023
:103480002100EFE710341022200004A908F0D0F842
:10349000029B013301D1069B0293882304995B05AB
:1034A000C918059B06981A03120B049105928142D4
:1034B00003D02B4201D107F08BFF019B013B01930D
:1034C000019B002BDED1029B002B03D004930498B8
:1034D0004168084709B030BDE025014C2D03EFE7F6
:1034E0000000011150485936F7B50F490F4B0A68D3
:1034F00004001A4084235B0013430B60030003277E
:103500001033019300252E00112008F001F8084B1C
:103510001B683B40AB4002351E43202DF4D1019B7C
:1035200040C4A342EED1F7BD5CF0004000FEFEFFB8
:1035300064F00040802270B5AD4CAE4BD20000214B
:1035400020001C6008F074F92300AB4A88331A602D
:10355000AA4B1A786E23002A00D01133E3620A23A3
:103560002365A74B1878A74BA0630138E361C3B26A
:10357000032B01D810232362A34B37226361C82396
:10358000DB00A36123008C331A60082336210F3A35
:10359000E518E16323646264E9670439251DE9677E
:1035A00025003B26BC352E602500C0352B6025004C
:1035B000C4352A6025000636CC352E602500083E2D
:1035C000C8352E602500D03529602100D4310B602C
:1035D0002100D8310A6021000225E0310D6025006C
:1035E0004221DC35296025001B3EE4352E60250094
:1035F000E8352B602500EC352A6022000525F432E1
:1036000015602200F03211602200183190321160F2
:1036100022009432136023003C2298331A60AF23B7
:10362000DB002360794B2363032805D808F038F9C1
:10363000330235371523636096232100FA225B009D
:10364000A360E360C8332361714BFC319200A36433
:103650000A6062626F4A704DA2627322E2656D3A3F
:103660006265A2650232E5644A60022161669621C4
:103670008900A166626709210022E166A2676749A5
:10368000674A684E2167E2673560032811D808F061
:1036900007F996089EA61023CDE70E23CBE70C234F
:1036A000C9E720001A259C30056020000735A030AE
:1036B00005602000A83003602300FA20F833800062
:1036C000186023006420A433186023005F38AC33F3
:1036D000186023000338B03318602300C630B433B9
:1036E000186023000020B833186023003825FC330D
:1036F0009D604D4D5A665D644C4D9A64DD61962522
:10370000AD001D624A4D9A675D62F53DFF3D9D62C9
:103710001E25484ADD6618675867D9651966DA6755
:10372000BE23C021444A5B00E250444B4900635031
:1037300004316250C4225200A350FA23E4205B00FB
:103740000432A3500432A3503D493E4A3E4BD1605F
:103750003E49800019503E49E938FF3819503D492B
:10376000043019503C491038D1613C4911633C493F
:1037700051633C4911603C49195019003B48F831EC
:1037800008603B49D16582213A4A89005A501A00A3
:1037900039490832D1671A003849B432116088219A
:1037A000374A89005A501A00364988321160364A21
:1037B000DA6407F005FE012007F01AFE70BD200054
:1037C00014259C30056020000435A03070E72000EF
:1037D00010259C30056020000335A03068E72000EC
:1037E0000E259C30056020000235A03060E7C04601
:1037F0000004FF1F6866FF1F6071FF1F2846FF1F40
:103800004A0AFF1F3A07000080C3C9019A0200005C
:1038100050C300006A180000280A0000204E000073
:1038200088130000F009FF1F00400011681000001D
:10383000C4090000DC05000040420F001027000012
:10384000FD1BFF1FFC00FF1F0000FF1F2D2FFF1F90
:103850005532FF1FED30FF1FE11FFF1FFD1FFF1F30
:10386000A921FF1F491FFF1FCD28FF1F952CFF1FF8
:10387000D918FF1FD927FF1F4125FF1F4D25FF1F07
:10388000491EFF1F011FFF1FC11DFF1FF7B50B0CB6
:10389000FF270122009300233C001E001D009446D8
:1038A000019089B262469A401000084018413618CB
:1038B000B6B2FF2F02D1012E00D19FB20098024074
:1038C0001A41AD18ADB2FF2C02D1012D00D19CB22E
:1038D0000133102BE6D10320012E07D1012D04D195
:1038E000019B2401E4191C700138FEBD102EFCD18F
:1038F0000238102DF9D00230F7E710B5064C2378C6
:10390000002B07D10548FFF7EFFD0548FFF7ECFD59
:103910000123237010BDC0462866FF1F3C66FF1FB1
:103920002C66FF1FF0B58BB00D000123019010290C
:1039300036D8FFF7E2FF00231A001B48C15C0133B1
:103940005218102BFAD1023B002A29D0174B184CE1
:103950001F68002306A9E25C1600FA5C56405E541C
:103960000133102BF7D102AA07F0B2FF2A0002A9F7
:10397000019807F0BDFD07F0EBFE23681B182360DC
:1039800007F0E6FE63681B18636007F0E1FEA368BA
:103990001B18A36007F0DCFEE3681B18E36000233C
:1039A00018000BB0F0BDC0463C66FF1FC844FF1FA7
:1039B0002C66FF1F0223F0B501245F4D5F4E2B7074
:1039C0005F4B91B01C705F4F0393336808207B708E
:1039D00006F072FA0023984205D07A78552A02D070
:1039E000332A00D09CE03360002006F0E5FC07F0AD
:1039F000C7FCFFF79FFD07F0FBFE1F2201240021FB
:103A0000514B10AE1A70514B1C70514B1970514BE9
:103A100019689143163A0A431A6060221968914363
:103A2000403A0A431A6007F01BFF07F021FEC1204D
:103A3000FF21494B80001A588A431A50C522920030
:103A400098588843BF3901439950985843490840D2
:103A50008021C9010143802099509958C00509026D
:103A6000090A0143995080213D48490107F0B8FDFA
:103A7000032322003B49019400933B4807F058FD83
:103A80002C223A4905A807F0A3FC05AC6178207800
:103A9000023406F031FAA642F8D10121002006F0E6
:103AA0003FFB0121092006F03BFB314B314A1968ED
:103AB00003201140A022D2020A431A608022196812
:103AC00092040A431A6019682B4A1140802292031B
:103AD0000A431A60294B2A4A934200D8012007F072
:103AE00067FC07F05DFE07F0D3FC287807F020FEA6
:103AF000039B1878C0B207F04BFD07F0B9FE2149CF
:103B0000042007F0ADFD06F023FC00F0AFF800F054
:103B1000EFFD00F081FE00F019FA002011B0F0BDB9
:103B200000932100174A042007F092FC8023DB0554
:103B30009C62FFF783FC57E74A0AFF1F34F00040FE
:103B40002846FF1FC463FF1F480AFF1F490AFF1FC3
:103B5000680AFF1FBCF0004000E100E0FF00FFFF2B
:103B60002C46FF1FB058FF1F2C56FF1FB0B9001185
:103B700014F00040FF7FF8FFFFFF9FFF6071FF1F01
:103B80000080FF1F3B00010870B500252849294A25
:103B900029484D6308CA1B051B0DED188242F9D157
:103BA0000022264B8B63264B08211A628022254B6C
:103BB0009205DA67244BDA688A43DA60234A12787E
:103BC000012A03D09A6822490A409A600121EE2412
:103BD0002048E40002686C438A430260DA681120DE
:103BE0008A43DA6007F0E4FC112007F069FC112039
:103BF00007F0A6FE184A200C0400642390420AD85D
:103C0000FA220023D200904205D9144B0A21C01891
:103C100007F076FCC3B2124A1372124BD4801B78A1
:103C2000002B04D1104B1021187807F049FE70BD0D
:103C3000000005408805054000060540FF01000022
:103C400000F0004004E100E03CF000404A0AFF1FA1
:103C5000FFDFFFFF00380040B70B000030F8FFFF28
:103C6000AC63FF1FE865FF1FE463FF1F002210B570
:103C70001100112007F034FE10BD0000F8B500233C
:103C800001250826394F3A4C3B62E3681120AB43CB
:103C9000E360E368B343E36007F012FC112007F030
:103CA00087FC112007F0ACFD402322682900134354
:103CB000236080236268DB02134380226360A36871
:103CC00007201343A360A3682A4A1340A3608023FC
:103CD000A2689B0113431022A360236C93432364C7
:103CE000236C2B43236480235B003B62226B224BBB
:103CF0001A402263626B1A406263A26B1A40A2638D
:103D0000E26B1340E3631D4AE3681340E36006F08F
:103D1000D9F92900072006F003FA8021184A11205A
:103D2000536C0B43536407F0C3FCFD21154B164A3B
:103D300089005A508023C720626B5B03134363637F
:103D4000E36880003343E360E368104A1D43104B8F
:103D5000E56019581140802212020A431A5080224D
:103D600092051A600B4B5E63F8BDC04600F0004040
:103D70003CF00040FFFFDFFFEFFFEFFFFFFF7FFFA3
:103D8000003800400000FF1F893B0011FF00FFFFCB
:103D900000E100E00000054030B503A804880B20D6
:103DA000002C0ED14968074D087849780902014373
:103DB0000A20A94205D1012120001980024B1B7A5B
:103DC000137030BD192A0000AC63FF1FF7B5150052
:103DD00008AA16884A680F4F1478527812022243B4
:103DE0000A24BA4214D10122DBB2019200962A00C1
:103DF00007F0FEF9041E0BD1074B1B68002B07D000
:103E000068782A78000210434242504101309847B6
:103E10002000FEBD022900003063FF1F30B50125E0
:103E200003790400BFB02B4212D00A49408806F043
:103E30004BFD28420CD06A46074B69465B8D558086
:103E40001380064B60881B7A1371002203F01CFE5E
:103E50003FB030BD2863FF1F7042FF1FAC63FF1FE0
:103E600010B50549054806F0E5FC0421044A05485B
:103E700006F0A2FC10BDC0462863FF1FFFFF000034
:103E8000DCB900117042FF1F10B5024804F07EFC3F
:103E900010BDC0461D3E0011062310B583701033BF
:103EA0000371443B43712A3383714433C37100234C
:103EB0000222012103720E4B027041701C88817234
:103EC0004472197A0273C1729A784273DA788273F3
:103ED0000322C2731A7902745A7942740C228274D2
:103EE0009A79C274DB7903751123C370152010BD54
:103EF000AC63FF1F10B5142007F032FB124B1422E5
:103F00000021186007F094FC002007F031FA01202E
:103F100007F0AEFA022007F0DBFB032003F0DAFE25
:103F2000042005F0EFFE052003F018F9062003F049
:103F3000E5FD072001F07AF9082006F01DFC0920B4
:103F400000F05CFF10BDC0463463FF1F10B507F0E2
:103F5000EFFC012007F09CFB07F072FA002010BD77
:103F6000094B10B50400984205D0012904D1200066
:103F7000064906F05FFC10BD0229FCD1013904F0AE
:103F8000C3FB0028F3D0F6E7FEFF00005A63FF1FD3
:103F900070B50D7A100004AA2C0016881022144067
:103FA000154220D1002E20D10A78022A18D14A6861
:103FB000517815780E4A09022943914205D00D4ADD
:103FC000914209D01C800A2404E014220A491A8074
:103FD00007F0FEF9200070BD0C2208491A80F7E7AF
:103FE0001C800124F6E70824F4E70B24F2E7C0461E
:103FF000F3FF0000F4FF0000AC44FF1FBCBA001147
:1040000010B504000749084806F014FC074804F0FE
:10401000FDFA0020E40704D50721054A054806F00B
:10402000CBFB10BD5A63FF1FFFFF0000613F001173
:1040300020BA0011B442FF1F00B50C4BBFB01A7874
:104040000B4901A800F01AFC6B4680B2588000288A
:1040500009D06A46074B69461B881380064B00222D
:10406000188803F011FD3FB000BDC0463863FF1F44
:104070003963FF1F0E43FF1F0E44FF1F00B50C4B9B
:10408000BFB01A780B4901A801F044FC6B4680B21E
:104090005880002809D06A46074B69465B8D13801B
:1040A000064B0022188803F0EFFC3FB000BDC0466D
:1040B0006263FF1F6363FF1FB442FF1F0E44FF1FB5
:1040C000F7B50E00377A1C0008AB11003D001A88C6
:1040D00020231D401F423CD13378022B3BD1736813
:1040E0001F785B781B023B431E4FBB4208D01E4F1C
:1040F000BB4214D01D4DAB4221D00A252800FEBD85
:10410000002A2AD1142C2AD82200F06807F060F97E
:10411000174B1C70012CF1D9FFF7B0FFEEE7002A16
:104120001BD1202C1BD82200F06807F051F9114B4D
:1041300004211C70104B187807F0C2FBDEE7E3B2D5
:104140000124009201940A00310007F051F80500A3
:10415000D4E70825D2E70125D0E70B25CEE70D25CA
:10416000CCE7C046F3FF0000F4FF00000229000086
:104170006263FF1F3863FF1FE463FF1F332310B523
:10418000040003700A220749013007F021F9064BA9
:104190000F201B681A0AE37222731A0C1B0E62733B
:1041A000A37310BDAC63FF1FD463FF1F30B501259F
:1041B00003790400BFB02B4213D00B49408806F0AE
:1041C00083FB28420DD06A46084B01A81B88138048
:1041D000FFF7D4FF6B46588000226946608803F0E1
:1041E00053FC3FB030BDC0465A63FF1F0E43FF1F54
:1041F00010B5024804F0CAFA10BDC046AD41001126
:1042000070B5160004AA148805AA15784A68507873
:10421000117800022A4A0843801805284BD807F075
:104220003FFB03131E29343F0720042C0BD8052223
:10423000121BAA4200D92A0022491A80300009190B
:1042400007F0C6F8002070BD0720112CFBD8122201
:10425000121BAA4200D92A001B491A80EEE7072048
:104260000E2CF0D80F22121BAA4200D92A0017499F
:104270001A80E3E70720032CE5D80422121BAA4288
:1042800000D92A0012491A80D8E70720032CDAD86F
:104290000422121BAA4200D92A000E491A80CDE737
:1042A0000720032CCFD80422121BAA4200D92A00CF
:1042B00009491A80C2E700220A201A80C3E7C046D3
:1042C000DCD5FFFF6BBA00118063FF1F5BBA0011E2
:1042D00056BA001151BA00114CBA001110B50D2197
:1042E000024A034806F068FA10BDC04640BA001101
:1042F0002443FF1F37B5002000F0CCF8204D214BA0
:10430000EA89287C9A422AD1042201A900F076F990
:10431000040000F033F9002C30D16B4699882B68EB
:10432000C9BA4B432989184A1B145B1853806B4642
:10433000D9886B6849BA89B24B4369891B0C5B18F1
:104340001248191C1BB2834200DD011C0B0400D56E
:104350000021138891800133138020003EBD022389
:10436000002101AA00F01CF96A4604000223012181
:10437000287C063200F014F90443CAE70124ECE774
:104380009463FF1F83050000AC63FF1F0F2700002D
:1043900037B5012000F07EF81F4D07226946287CC2
:1043A00000F02CF9041E33D16B461B787F2B2FD8DD
:1043B00000F0E4F86B46D878F02302041B031A409F
:1043C0006B469B8815495BBA9BB21A432B68000960
:1043D00053432A891B0C9B184B806B465A789B7859
:1043E00012031B011A436B68024353436A891B0C77
:1043F0009B180B481A1C1BB2834200DD021C1304DD
:1044000000D500220B888A8001330B8020003EBD3E
:1044100000F0B4F80124F9E79463FF1FAC63FF1FB9
:104420000F27000010B50F4C237C002B0CD0382B2D
:104430000BD1012000F02EF8CC22AC21207C92017F
:1044400000F028F900F09AF810BD074BE2899A4273
:10445000FAD1012000F01EF80021207C00F0FAF8CB
:10446000F0E7C0469463FF1F8305000010B5084BBA
:104470001A7C002A09D05B69002B06D09847041EDD
:1044800001D0FEF7BDFD200010BD0124F9E7C046B4
:104490009463FF1F70B500210600162005F076FE1C
:1044A0000121152005F072FE07F0AAF8040009208A
:1044B00007F0A6F900222B4B2B4DDA6661321A6009
:1044C00019685B3A9143002E28D0023A0A431A60D9
:1044D000AC4209D10A22DA6107321A6200221A6359
:1044E0009A630132DA6370BD204A944203D11E22DE
:1044F000DA610532F1E71E4A944203D13022DA61D3
:104500000632EAE71B4A944203D14322DA610832B9
:10451000E3E7194A9442E1D16922F7E702220A430C
:104520001A604622AC4203D0104A944204D194222D
:104530005A6106329A61D1E70D4A944201D1E622CE
:10454000F6E70C4A944204D13422FF325A610D320C
:10455000F0E7094A9442C1D1E62252005A610A3278
:10456000E8E7C046005000400024F4000048E8019D
:10457000006CDC020090D00300D8B80510B5002410
:10458000064B0920DC6606F09BFF2100162005F093
:1045900099FD2100152005F095FD10BD005000404B
:1045A000F8B51C000023134D0F00EB666860160081
:1045B00007F016F901238022EB6623002F615200D9
:1045C000013B08D206F0A4FE08200B4A1168002C1B
:1045D00003D12000F8BD2A61F2E72B6F034203D01C
:1045E0002B69013C3370013613685B1A032BEED93B
:1045F0000124EEE7005000406008FF1F002370B563
:10460000124D1400EB6668600E0007F0E9F8012314
:104610008022EB6623005200013B08D206F078FEB0
:1046200008200B4A1168002C03D1200070BD2A61BC
:10463000F2E72B6F034203D02B69013C3370013644
:1046400013685B1A032BEED90124EEE700500040FB
:104650006008FF1F002370B50C4C0D00E36660601E
:1046600007F0BEF80123E366256106F051FE8020C5
:10467000074A80001168636B034205D113685B1A17
:10468000032BF8D9012070BD0020FCE7005000404A
:104690006008FF1F002370B5134C0E00E3666060D6
:1046A000150007F09DF80123E36626610F33626B66
:1046B0001A42FCD02B0A23611023626B1A42FCD0F1
:1046C000EDB2256106F024FE8020084A80001168C2
:1046D000636B034205D113685B1A032BF8D90120E1
:1046E00070BD0020FCE7C046005000406008FF1F7E
:1046F00010B5084CE368002B08D1074B1B685B041E
:104700005B0C0A336360054B1B68236006F008FFEF
:10471000A06010BDD463FF1FC8F00040CCF0004083
:1047200010B507F05DF80F4B996A9A6A8A42FBD17F
:104730000D4C6268A0688A18121A531E884200D372
:104740001300A1602168DA0B52185B0407495B0C67
:10475000636022600B60064B1A6006F0D9FD20688A
:1047600010BDC04600F00040D463FF1FC8F00040F9
:10477000CCF0004070B51F4C23793F2B01D93F236B
:1047800023711D4B22791A701878C0B206F078FF99
:1047900018231A491A4A0B801A4913800B80538038
:1047A000A379194980200B800C21938001334B435E
:1047B0000001191C834200D9011C144BD1801980BF
:1047C0006379002B11D101336371237A012B01D856
:1047D000022323726279237A0D4853430A215843F6
:1047E00006F08EFE0B4D286070BDA02BEDD9A023E6
:1047F000EAE7C046C863FF1F480AFF1F0C44FF1FBB
:10480000D445FF1F0A44FF1FB465FF1F0844FF1F64
:1048100071020000B863FF1FF8B512210020FEF7F7
:10482000D5FD114C011E114D09D10C22104BC1CBED
:10483000C1C4280006F0FCFFFFF79CFFF8BD0C2266
:1048400020000C49FEF796FD0C2802D0084B43CB04
:1048500043C40C2228000849FEF78CFD0C28EBD03D
:104860000C220021E5E7C046C863FF1F9463FF1FC9
:10487000B0BA0011FC0C0000F50C0000F0B50025EA
:1048800004000E0085B0AA4263D04B1C0878019347
:104890004B788978377909021943F3783F061B046E
:1048A0000B431F43039720706570252800D173E0E8
:1048B00012D810280AD806F0F3FF46E52C2C2C87D6
:1048C000958E2C2C2C2C2C2C2C2CC500232800D184
:1048D000A7E0FF23637094E0562857D010D8332800
:1048E00000D199E0552837D02628F2D1934B2900E2
:1048F000132218001D0006F09BFFFEF781FB5AE013
:10490000722800D17FE0DC2800D1DAE0712800D1E4
:104910006FE0DB2800D0EFE0042ADAD91025052A61
:1049200005D0551F2A003800711D06F051FD0522E3
:104930003100200006F04CFD2A003900601D06F011
:1049400047FD053505E00C2220007D4906F040FDBD
:104950000C25280005B0F0BD013A7A4D0C2A13D879
:10496000002A0AD02800019906F032FDFFF702FF65
:104970000C2228007449FEF737FC29000C22601C29
:1049800006F026FD0D25E4E70C22EBE76D4D6F4B9D
:104990002A0043CB43C2E9E7013A684D0C2A11D8FB
:1049A000002A08D00199280006F012FD0C222800E8
:1049B0006749FEF719FC29001322601C06F008FD68
:1049C0001425C6E70C22EDE705226249601C06F0BB
:1049D000FFFC0625BDE712225F49601C06F0F8FCCB
:1049E0001325B6E708225D49601C06F0F1FC092595
:1049F000AFE77178F72900D96BE7594B188801F0B8
:104A0000E5FB0225A5E7574B012A03D072781A70FF
:104A10006270F6E71B785DE72000FFF7AFFB05004B
:104A200097E7042A04D9504D2F6006F079FDA8605D
:104A3000FFF776FE0422039003A9601C06F0C8FC71
:104A4000052586E7494D062A15D906222800019931
:104A500006F0BEFD00280ED006220199280006F0BF
:104A6000B7FC062242492800FEF7BEFB01233D4A5F
:104A700011780B43137029000622601C06F0A8FC75
:104A8000072566E7931E3B4F1A2B04D87378002B3B
:104A900009D100F027F9384B39001D78601C6A1ED7
:104AA00006F096FC55E7551E2A000199380006F0DD
:104AB0008FFC3249AAB23800FEF796FB00F048F9A5
:104AC000E9E7022A00D804E77378BFB26370B378CD
:104AD000A370032A05D0033A390092B2F01CFEF706
:104AE00083FB10223900E01CFEF744FCC51C0028A3
:104AF00000DB2EE7607084E7DA2800D0E9E6042ABC
:104B000000D8E6E6082A15D9B37972791B02134357
:104B1000F27912041A43337A1B0613433B603B6855
:104B2000052231002000039306F052FC0422601D90
:104B300003A95AE7FE236370F1E7C0469463FF1FA1
:104B4000BCBA0011C863FF1FFC0C0000B0BA001112
:104B5000F50C0000A063FF1F8063FF1F4845FF1F87
:104B60000E44FF1FC463FF1FD463FF1F6509FF1FAF
:104B7000ADAC0000C765FF1FC565FF1FAEDE0000BE
:104B800070470000020010B5094B0A32094C92B27E
:104B9000DA815A8298811882207802F07DF9042205
:104BA000054B012120781A7006F08AFE10BDC04620
:104BB000D244FF1F1266FF1F1166FF1F013870B538
:104BC000042809D806F06CFE0309230812001E4BC6
:104BD0000221187806F074FE70BD1B4B082118786E
:104BE00006F09EFB0022194B1A72F5E78022002482
:104BF000164B154D52001A81082128781A68DC726C
:104C000006F0FEFB2100287806F07AFDE4E70E4B63
:104C10000821187806F084FB0D48FFF73DF90D4B8D
:104C20000D4A9B7993800D4A13800022074BDA725C
:104C30000132FF321A810A4B1B78002BCCD0094A73
:104C4000136006F0FDFCC7E7E463FF1FB863FF1FB6
:104C50001744FF1FC863FF1FD445FF1FB465FF1F24
:104C6000C463FF1F34F0004010B5002905D10828A7
:104C700003D10131013005F053FA10BD10B50129FF
:104C80000FD108280DD10021013005F049FA054B5C
:104C90001B78002B05D02622034B04485A72FFF7DD
:104CA00071FF10BDE865FF1FB863FF1FC409000056
:104CB0000300F0B50A4D8E18B14202D1520080189F
:104CC000F0BD0C782F6824093C5D0F271C700C7810
:104CD00001313C402F683C5D5C700233ECE7C0461C
:104CE0000444FF1F0E22114B10B51A700D23104CF7
:104CF00010492370093A043B0F48637006F068FBC3
:104D00002D2301220D490E48E371FFF7D1FF012247
:104D10000C49FFF7CDFF01220B49FFF7C9FF002225
:104D20000A491000FEF760FA10BDC046E465FF1F97
:104D3000C565FF1F6BBA0011C765FF1F6709FF1F1D
:104D4000CD65FF1F6609FF1F6509FF1FAEDE00006E
:104D500070B5124C132220001149FEF70BFB114DC8
:104D6000002817DDAB78002B14D0431C2B700923CF
:104D70006B70002300190370287829000130C0B23D
:104D800006F04EFC297822000139C9B2002005F056
:104D900031FC70BDFFF7A6FFEEE7C046C765FF1FF9
:104DA000AEDE0000C565FF1F10B5114B1A781870F4
:104DB000002A0ED000280BD10E4B1A78062A07D8ED
:104DC0005423D340DB0703D50B4B187802F064F86B
:104DD00010BD0028FCD0074B1B78012B02D0033BF1
:104DE000022BF5D8044B0121187806F069FDEFE796
:104DF000E865FF1F1166FF1F1266FF1F70B5504E5A
:104E0000504A51493070082005F080FA01210920EC
:104E100005F086F9092005F067FA0121002005F068
:104E20007FF9002005F060FAFEF7EAF806F0B8FB1B
:104E3000032246494648FFF73BFF2D240300042286
:104E40001C7044490130FFF733FF30230470424D9A
:104E5000424C437083702E3B062220004049EB8772
:104E6000FEF788FA062813D0200006F049FD022834
:104E700009D00321200006F0CBFB8D23E3706E3BAD
:104E8000237119336371062220003549FEF7ACF90E
:104E9000344B1B68FC335C64FFF75AFF0020FFF7BC
:104EA00083FF314C314A0121314B1278207801F0D7
:104EB000B5FF304A304B12780021207801F0AEFF68
:104EC00001222E4B1A702E4B5B78552B31D12D4B76
:104ED0003B325A722C4B2D4AAB81EA812B826A827B
:104EE0002021307806F0E4FC0120404205F0CEFBA2
:104EF0000120404205F06AFCFFF7F0F9FEF7B0FF31
:104F000000F0A0FC01204042FFF77AF8012006F0F3
:104F1000FFFBF72001F03EF90121307806F0D0FCCC
:104F2000307802F015F91A4806F05AFAFEF7A6FE94
:104F300070BD6422174B5B7953431A000A32CBE7EA
:104F4000E463FF1F694C00117D4C00114845FF1FB1
:104F50008063FF1FA063FF1FD244FF1F6509FF1F6F
:104F6000ADAC00006866FF1F1266FF1F3644FF1FCE
:104F70001744FF1FE465FF1FC565FF1FB665FF1FD0
:104F8000C463FF1FB863FF1FC4090000CE090000FF
:104F9000E663FF1FC863FF1FF8B50A0020230D005A
:104FA0001A40194251D0544B1B78002B3CD0FFF7CC
:104FB000B7FB524B524C534E99686268737A8A1A07
:104FC000DB039A4202D36160FEF758FE327A217AFF
:104FD000531EDBB299422AD1FFF724FA637A002BE1
:104FE0001FD0013BDBB26372002B1AD1464B5B78BA
:104FF000552B01D106F024FBE37A002B0CD00023C3
:10500000424A434FE3721388380001331380FEF79E
:1050100043FF390006F04CFA642370795843FFF7D8
:10502000B1FD237A0133237220206840F8BD9142FC
:10503000D4D300232372FFF719FA354F3800FEF757
:105040002BFF390006F034FAC8E70BB2002B0ADA5E
:10505000304B187806F07CFC002801D006F080FB6D
:1050600080200002E1E70224214206D0244B0120E7
:105070001A72FFF799FE2000D7E70B071BD5FFF741
:105080004FFB1E4B1E491F4C98684A68637A821A70
:10509000DB039A4202D34860FEF7F0FDFFF7E6F922
:1050A000FFF7C0F900F0E8FB2368DB0701D5FFF745
:1050B0009FF80820B9E710240E002640214206D0B0
:1050C0000D4B1B78002BD6D1FEF7DEFED3E7012473
:1050D000214209D0104800F06DF806F0B1FB310014
:1050E000092005F01DF8C6E70424080020402142ED
:1050F0009CD0FEF7A1FFBEE7E865FF1FD463FF1F4A
:10510000B863FF1FC863FF1FC463FF1FAC63FF1FAB
:105110001744FF1FE463FF1FFC43FF1FF0B51B4B49
:105120001B4F1B883A8804001A4E1B4D85B09A42CB
:105130000DD832889A420AD3184B1A882B889A4283
:1051400005D1174A174B12881B889A421BD005209D
:1051500001F076F83B8802AA1380338801905380CF
:105160002B88114D93800F4B02A91B88D3800F4BC6
:105170002A78188802F092FD0D4B08212878019AB0
:105180001C7006F005FC05B0F0BDC046B265FF1FFF
:105190000C44FF1F0A44FF1FB465FF1FB065FF1FCB
:1051A000AE65FF1F0844FF1F1266FF1F0E44FF1F5E
:1051B000AC65FF1F13B50C4B1C78002C11D10028D7
:1051C00001D00A4B18600A4A0A4B11780A4A107833
:1051D0000A4A01920A4A0092002205F003F92000CF
:1051E00016BD1124FBE7C0461166FF1FA865FF1F0F
:1051F0001066FF1F0066FF1F1266FF1FEC65FF1F92
:10520000F065FF1F10B5064B12201B78052B06D149
:10521000044B13221988044B187801F0EDF910BDE6
:105220001166FF1F0E44FF1F1266FF1F10B50024FA
:105230000122114B52421870104B1C70104B1A80F7
:1052400001F086FF04220F4B21001A700E480C3229
:1052500006F026F9102221000C4806F021F9072259
:105260000B4B1C600B4B1C700B4B1C700B4B1A70C8
:105270000B4B1C7010BDC0461266FF1F1166FF1F4E
:105280000E44FF1F1066FF1F0066FF1FF065FF1F23
:10529000EC65FF1FC465FF1FC365FF1F1044FF1FA0
:1052A000C265FF1FF8B5174C0600257806A8142420
:1052B0000078052D23D1B41F134FA5B21824BD4289
:1052C0001DD88D1FADB2BD4219D8FA256D00AA4276
:1052D00015D21D000D4F0A3DADB2BD420FD80C4C8A
:1052E00026800C4C21800C4900240A800B4A138034
:1052F000FFF714FF0A4B0421187806F011F820007C
:10530000F8BDC0461166FF1F790C0000750C000047
:105310000C44FF1F0A44FF1FB465FF1F0844FF1F12
:105320001266FF1FF0B50BB20D0089B0002B00DB39
:1053300070E1A44E307806F00BFB041E50D00378C9
:10534000A22B00D122E1D02B1AD0912B45D143784A
:105350000E2B42D19C4B82889A423ED19B4A836855
:105360001278052A39D1032018567F2835D0984B5A
:105370001B68002B31D05B68002B2ED098472CE0A7
:105380008078072829D806F08BFA0428183F3F7444
:10539000A8D86378002B0CD101218C4B19708D4B50
:1053A0001A78002A5BD08C4B307801F037FD00284A
:1053B00055D00722854B1A7051E061780029F8D149
:1053C000E378002B11D0854A854B1278307801F0B4
:1053D00025FD60706378002BEBD1200006F0C0F94A
:1053E00080200002684009B0F0BD784B1B78022B8A
:1053F000F3D00121307806F073F80028EAD10121BA
:10540000307806F05DFAE5E76378002BD1D16F4F75
:10541000032807D13B78052B02D101333B701EE0F6
:105420000223FBE76F4B1A886F4B0293002A0BD0C5
:105430001B78002B03D00121307806F0A9FA3B78C5
:10544000062B04D1013BE9E7029B1A70F7E7042B16
:1054500041D10121029B3078197006F031FA5C4B82
:105460001B68002BB9D01B68002BB6D0574A1078A8
:1054700084E76378554F002B27D10622211D5B4816
:1054800005F0A6FF62895A4B5A491A80A2895A4BE5
:105490001A80E3890B800521397058490A80584ADF
:1054A0001380228A574B1A80574B1B78012B09D146
:1054B0001F2000F0C5FEFA229200424304213078FA
:1054C00006F066FA0022484B75E7312B00D070E7F2
:1054D0000022454B1A700323A0E70622002143480F
:1054E00005F0DEFF0023454A04211380444A30784A
:1054F0001380444A138005F013FF0821307805F02B
:105500000FFFA379083B5A425341304A03331370CB
:10551000304B1B78002B06D0334B30781A78002A9A
:1055200006D001F0B9FC0122314B52421A8096E7B5
:105530000121197006F0C4F9F5E70821307805F06B
:10554000EFFE6378002B00D047E72C4B2D4F0293E2
:10555000E388029A04211380294B3078039323892E
:10556000039A138063893B8005F0BAFF002800D0BE
:1055700033E7264B1B68002B00D12EE703990298D6
:105580003A88098800881B68984726E74379132BD7
:1055900000D022E70389012B0AD11D4B1B78022B77
:1055A00006D10821307805F0BBFEFFF72BFE14E78B
:1055B000052000F045FE08210200307806F0E8F9E9
:1055C0000BE7C0461266FF1F051400001166FF1F9F
:1055D000A865FF1F3644FF1F1744FF1FE465FF1F28
:1055E000C565FF1FE665FF1FE865FF1FB765FF1F65
:1055F0000E44FF1FBE65FF1FC065FF1FB265FF1F82
:10560000B065FF1FAE65FF1FB665FF1FA465FF1FD6
:10561000AC65FF1F8020C001014200D0E2E6CB074D
:1056200031D5324B1B78002B1DD0314E05AC337871
:10563000052B1AD1023B23702E4B21001B782372BD
:105640002D4B1B7863722D4B187801F08BFB0028D3
:1056500009D007202A4B30701B68002B03D01B6831
:10566000002B00D098470120BCE60E20254B0622D7
:105670001B7825492370254B1B78637002ABC0183B
:1056800005F0A6FED8E7022308001840194209D009
:10569000174B1B78052B03D11D4B188806F028F8F3
:1056A00002209FE60424214203D0FFF737FD2000AB
:1056B00098E6082308001840194200D193E6154BDC
:1056C0001C78012C03D0022C0DD008208AE6124B46
:1056D000124A134913481B881288098800880094CD
:1056E000FFF7E0FDF1E7FFF78DFDEEE7E865FF1F4F
:1056F0001166FF1F1044FF1FC265FF1F1266FF1FC8
:10570000A865FF1FC465FF1F1144FF1FC365FF1F6E
:105710000E44FF1FAC65FF1F0844FF1FB465FF1F49
:105720000A44FF1F0C44FF1F10B502A804880B2079
:10573000002C10D1496808784978090201430C48C7
:10574000814209D1022119800A4B59881170DB78F6
:1057500000205BB2537010BD074C0A20A142FAD161
:1057600002211980034B998811705B79F0E7C046DC
:105770006E2A0000AC63FF1F6F2A0000F7B515000A
:1057800008AA16884A680F4F1478527812022243EA
:105790000A24BA4214D10122DBB2019200962A00F7
:1057A00005F026FD041E0BD1074B1B68002B07D00C
:1057B00068782A78000210434242504101309847ED
:1057C0002000FEBD022900002466FF1F30B5012520
:1057D00003790400BFB02B4227D01549408805F05B
:1057E00073F828420DD06A46124B69465B8D1380D0
:1057F00002235380104B5B8893806088002202F064
:1058000043F90E49608805F05FF8C0070DD56A4678
:105810000B4B69461B88138002235380064B9B88E1
:1058200093806088002202F02FF93FB030BDC0465F
:105830001C66FF1F3844FF1FAC63FF1F1466FF1F69
:105840009244FF1F10B5074C0749200004F0F2FFF7
:105850002000064904F0EEFF0721054A054804F040
:10586000ABFF10BDFFFF00001C66FF1F1466FF1F8B
:105870003CBB00113844FF1F10B5024802F086FF00
:1058800010BDC046CD5700110200F0B501270A48EF
:105890000A4E51188B1A002B00DCF0BD0824157835
:1058A0004308684038404000805B013C58406D0828
:1058B000002CF5D10132EDE7FFFF000056BB0011CF
:1058C000F0B500250F269D4200DBF0BD4C5D0709B9
:1058D00044403440A400A05801357840F3E700006C
:1058E000F0B589B06A460D000B000F271100103586
:1058F0001C780133260024093E4016705470023291
:10590000AB42F5D12023024AFFF7DAFF09B0F0BD20
:105910005CBB0011F0B54E780B7889B036020C00F4
:10592000170001901E43012A61D9954B9E4200D871
:1059300077E001339E421CD1062A17D1CA788B78B2
:1059400012021A430B791B0413434A7912061A43B5
:105950008C4B5A6100221A705A808B4A5A608B4ACB
:105960009A608B4ADA60002009B0F0BD88225205A7
:10597000EEE7884B9E423CD182498B78002B00D0C9
:10598000F6E00C2A31D10F22A3789343E278120279
:1059900013432279120413436279120613434B60B6
:1059A000E279A07912020243207A00041043627A5D
:1059B00012060243CA60E27AA07A120202437648D3
:1059C0004A81834208D804236E49142201980B703F
:1059D00005F0FEFC1420C7E71201D21889235B05ED
:1059E0009A42F0D801238B70BDE7022AFAD0052332
:1059F000EAE76A4A01239642E6D1FFF703FC052F46
:105A00000CD9E378A2781B021343227912041A43BB
:105A100063791B061343624A0393136005F010FE7B
:105A2000A1E7584D2B78002B9DD1AB78002B00D1EE
:105A3000A0E02B8901339BB20093B34200D091E0E8
:105A4000132AD4D9CF7C8B7C3F02122120001F4324
:105A5000FFF71AFF874200D08EE0002E3DD1E37899
:105A6000A2781B0213432279E96812041A4363796E
:105A70001B06134303930A228B4212D1FF23A37008
:105A8000E370237163716B89002B09D1E37B227C66
:105A90001B0212041343A27B13431B0901336B81C6
:105AA00000226B89002B8ED0002A67D168683701ED
:105AB0003818000B6B6900030390984205D96861A0
:105AC00005F0B6FCEB780133EB7068681022A11C7E
:105AD000381805F09DFC2E8145E76F89009A7B1EE2
:105AE0009BB293423AD1E278A37812021A43237907
:105AF00005A81B04134362796C6812061A43EB680D
:105B000000920392211D0C22049305F061FC0120F8
:105B1000260004A940421036FFF7E2FE013F012FA4
:105B200017D1009A0B232861824200D04CE704224F
:105B30001C49200005F06CFC042203A9686805F0EC
:105B4000FFFCE968039AFF23914200D13CE7F73B51
:105B50003AE73100FFF7C4FE1036DFE70923B7420A
:105B6000A4D831E7009BB34200D9FCE607232BE71A
:105B7000022329E7032327E7062325E70A2323E750
:105B8000FFFE0000AC44FF1F00000111FFFF0000FA
:105B90005048593601FF0000FFFF001102FF0000CE
:105BA00034F00040B844FF1F10B5034C0B00012235
:105BB000210000F06BFA10BD695D00110B8870B513
:105BC00006000D000224162B11D92B0003220949CF
:105BD00000F05CFA041E0AD1074B2A881B88191CA6
:105BE000934200D9111C300089B200F0EFFA200076
:105BF00070BDC046955D00118266FF1F10B54A78E2
:105C00000400013A0B000220012A07D80A78002A72
:105C100004D005222000024900F038FA10BDC04629
:105C2000C35D00110A7810B50B0004000220002AA1
:105C300004D007222000024900F028FA10BDC04617
:105C40006F5E00110A7810B50B0004000220002AD4
:105C500004D009222000024900F018FA10BDC04605
:105C6000D55E001110B5034C0B000B22210000F093
:105C70000DFA10BD055F001110B5034C0B000D228D
:105C8000210000F003FA10BD775F001110B5034C3E
:105C90000B000F22210000F0F9F910BDD15F0011B7
:105CA0000A7810B50B0004000220002A04D011224B
:105CB0002000024900F0EAF910BDC046E15F001182
:105CC000002310B51322190000F0E0F910BD000008
:105CD00010B5034C0B001722210000F0D7F910BDBE
:105CE00033600011002310B51922190000F0CEF91D
:105CF00010BD000010B5034C0B001B22210000F06A
:105D0000C5F910BD6D600011F7B584890D0006005E
:105D10000121002C22D000238268D3561778002B53
:105D20001EDA0C2C1AD90C3CA4B21319408800932B
:105D3000230002F086FE431E984101307B06DB0FF4
:105D40006B703F23013C1F40A4B22870AF70AC8041
:105D5000002C07D0B3680133AB6000210800FEBD02
:105D60000020EBE7AC60F8E70B7803704B884370DA
:105D70004B881B0A83700B79C37004207047042082
:105D8000022B06D10020537811781B02009A0B4396
:105D9000138070470B8803700B881B0A4370022026
:105DA00070470420009983420AD1537810781B026F
:105DB00003430B80D37890781B02034300204B8071
:105DC0007047F8B50D004B7801240021461C037084
:105DD0002B788B4201D82000F8BD6B78B01C4F1C8B
:105DE000012B10D1890069184B88022233704B882F
:105DF000B9001B0A7370691805F07AFB0436043485
:105E0000A4B2F9B2E4E7122359436B185A8804315B
:105E100032705B8810221B0A7370691805F068FBEA
:105E200012361234ECE770B5049D14001E00052BE9
:105E300001D8042070BD637812781B0213432B80B5
:105E4000E378A2781B02134302226B802A71211D82
:105E5000681D063E05F04CFBB2B22A81F02AE8D854
:105E60002800A11D0A3005F043FB0020E2E70023D3
:105E700010B50A789A4201D8900010BD9A008A188D
:105E80005488013304705488DBB2240A4470948827
:105E900084709288120AC2700430EAE710B51100CB
:105EA000029C062B04D004201022142B01D010BD1C
:105EB000022222714B7808781B0203432380CB789F
:105EC00088781B02034363800431601D05F010FBDA
:105ED0000020ECE710B50C788B7804315C43E4B219
:105EE00003702200013005F003FB601C10BD04208C
:105EF000022B06D10020537811781B02009A0B4325
:105F00001380704710B50C000A88023105F0F0FAD2
:105F1000208810BD70B504000D0004981100012BFD
:105F200001D8042070BD16785278120232430280E4
:105F30000200F83255701470E825002C00D10C35A1
:105F4000023B9AB24280AA42EBD80231043005F0FB
:105F5000CFFA0020E6E70420009983420AD1537863
:105F600010781B0203430B80D37890781B02034305
:105F700000204B80704710B50C000A88023105F0F4
:105F8000B7FA208810BD000070B501211E00042062
:105F9000049C0E400B4218D1CB40DDB28D4214D987
:105FA0000A49DBB2098899420FD32300F6331D70EA
:105FB0003300580011184978165C09023143013347
:105FC0002152D9B28D42F4D8002070BDCC44FF1FBD
:105FD00010B50C000A88023105F08AFA208810BD3D
:105FE00010B50C788B7804315C43E4B20370220066
:105FF000013005F07DFA601C10BD10B5110002984B
:10600000032B01D8042010BD14785278043B1202EF
:1060100022430280CA788C781202224342809AB2CC
:106020008280F22AEED80431063005F061FA0020B1
:10603000E9E710B50C000B8803700B881B0A43704E
:106040004B8883704B881B0AC3708A8804300631E2
:1060500005F04EFAA088043080B210BD0420012B58
:1060600003D100201378009A1370704710B50C000C
:106070000B8803700B881B0A43704A880230043176
:1060800005F036FA6088023080B210BDF0B589B0F4
:1060900003931E4B029242000700D05A019102F076
:1060A00020F81325061E2DD0029B01240370019BAE
:1060B000002B04D0001903999847001984B26B464D
:1060C0001B7A5BB2002B0FDA1021380002F01CFBA8
:1060D0001925002813D130003219E1B202F066FC14
:1060E000051E0CD10C34A4B2042304AA380005A95F
:1060F00093800696948101F0AFFD051E02D030001A
:1061000005F046F9280009B0F0BDC0468066FF1FC3
:1061100070B505000C0000280CD00020814209D089
:1061200010222000044905F0E3F901202B782373A5
:106130006B78637370BDC0469CBB0011F0B5060060
:106140000D0017001C0085B002291BD0002010296B
:1061500007D1022B07D0102B03D115E00020102C03
:1061600008D005B0F0BD69463800FFF7D1FF2A001E
:1061700069460BE069463000FFF7CAFF2200694616
:10618000380004E0022BE9D12A003900300005F084
:10619000DFF9E6E7031CF72800D9F72303200849B5
:1061A0009AB2013A0B80D317034006499B189B1003
:1061B0000B80D30F04499B185B100B807047C046BF
:1061C000D044FF1FCE44FF1FCC44FF1F034B1B884E
:1061D0008B4202D3024B4000C1527047D044FF1F94
:1061E0008066FF1F014B4000185A70478066FF1FF2
:1061F0001722014B1A8070478066FF1F70B505009B
:106200000E2005F02DF9041E13D0D02303700023B7
:106210000622837007494570033005F069F9064B83
:106220002100DA8A62811B7E2373044B187805F003
:10623000C7F970BD9C66FF1F8C66FF1F2045FF1FBE
:10624000262803D8024B4000C05A70470148FCE79B
:10625000D244FF1FFFFF000070B506000C00094D7F
:106260001C220021280005F01BF9074B1E70074B6C
:106270001C7005F06DF80123002801D000231220C6
:106280002B7070BD8C66FF1F2045FF1FAD66FF1F82
:1062900070B505000D4C0800E260A16010220021DD
:1062A000656005F0FDF9012803D11021A06802F016
:1062B00058FD10220021280005F0F2F9012803D131
:1062C0001021606802F04DFD70BDC0468C66FF1F56
:1062D00070B5041E05D1002903D006220D4805F033
:1062E00007F90D4B1D78012D11D1002C05D102228B
:1062F0001A7005F095FA280070BD00221A70074B3D
:106300001B78FF2BF7D02000FFF778FFF3E700257D
:10631000F1E7C0469C66FF1F8C66FF1F2045FF1FEC
:10632000030010B5002801D1002010BD00780B4AF1
:10633000002803D15988D1821B7913761378022B58
:10634000F2D10023984200D103331370044B1B7821
:10635000FF2B01D0FFF752FF0120E6E78C66FF1FFD
:106360002045FF1F002911D000280CD04B790128AF
:1063700003D140225242134303E03F22134003283B
:1063800002D001204B7170474022F4E70800FAE781
:1063900070B5094D0100287800280BD0074C062263
:1063A000200005F0A5F821002878FFF7DBFF20008A
:1063B00005F066FA70BDC046AC66FF1F8666FF1F1B
:1063C00000290AD0012808D13F224B799343C02BE2
:1063D00003D0403B5A425341981C704770B5174D4B
:1063E00006002B78FF2B15D00A2005F039F8041E83
:1063F00010D0D0230370C83B8370114B11491B7818
:106400004670C3700622043005F072F82100287827
:1064100005F0D6F80C4B1B78012B0DD10B4B1B68EC
:10642000002B03D09B68002B00D09847084B042119
:106430001878084A04F0E4FF70BDC0462045FF1FED
:10644000AC66FF1F8666FF1FA866FF1FD466FF1F8E
:10645000D866FF1F60EA0000014B98687047C0468D
:106460008C66FF1F014BDB68186870478C66FF1F46
:10647000074B10B5DA68136801331360054B1878C1
:10648000FF2803D08021C90105F01AFA10BDC046CB
:106490008C66FF1F2045FF1FF7B50E0002F0C8F8FD
:1064A000051E1CD00E4B06621F78002F00D1077806
:1064B000AB791020019304F0D3FF041E0FD0D0233A
:1064C0000380C73B8370019BE91DC3700622043023
:1064D00005F00EF821003800E66005F071F8F7BD10
:1064E0001E45FF1F014B18787047C046AC66FF1F62
:1064F000054B002805D1054B1A78054B002A00D121
:10650000014B18007047C0469C66FF1FAC66FF1F1A
:106510008666FF1F014B58687047C0468C66FF1F98
:10652000024B1868431E9841C0B27047B066FF1F07
:10653000421E03000120152A03D9FF3B5A42534152
:10654000D8B27047F0B51C0000230E0085B0039050
:1065500002920B70029A934201D3002019E0E55C8D
:106560005A1CD2B2002DF8D0029851198142F4DCA5
:106570000233DFB2A35C18000193FFF7D9FF0028B4
:1065800007D0013D019A0399EBB233708A4202D1E0
:10659000E01905B0F0BDDB19DBB2DBE710B50C008C
:1065A00002F09EF803001220002B03D0210058882F
:1065B00005F0C6F810BD000070B50E4D840063599B
:1065C000002B15D0186A002801D005F001F92B59CD
:1065D000586A002801D005F0FBF82B59986A00286A
:1065E00001D005F0F5F8285905F0F2F800232B51F9
:1065F00070BDC046BC66FF1F1C4B70B504000E008A
:10660000150099420AD11A4B1B68002B01D11220A8
:1066100070BD1B68002BFAD09847F9E7154B9942DB
:1066200015D1134B1B68002B0AD01B68002B07D019
:106630009847002804D1104B1C70104B1D70E7E7E1
:1066400029002000FFF7AAFF0028E1D1F3E70800A6
:1066500001F0EEFF0028DAD003780320A342D7D15F
:106660002900300005F06CF8D2E7C046FEFF0000BC
:10667000B866FF1FFFFF0000B566FF1FB466FF1F6F
:10668000F7B50400808801F0D3FF0025A84203D0AD
:106690000578A08802F008F81C4E3378002B1FD034
:1066A000AB421DD11A4B28001978FFF777FF00285D
:1066B00018D000233370A3790820A778A688019307
:1066C00004F0CEFE011E0DD0D0230370CA3B8370B0
:1066D000019B477086808371280004F071FF01E000
:1066E000002DE8D1A0880B4B8200D358002B01D09D
:1066F000FFF762FF1721A088FFF768FDA08801F06F
:1067000027FDA08801F0FEFDF7BDC046B566FF1F5E
:10671000B466FF1FBC66FF1FF0B587B01D000CAB51
:106720001B88070001930DAB1B88142002930EAB4E
:106730001B88160003930FAB1B880091049310ABCA
:106740001B88059304F08CFE041E1AD0D02303701E
:10675000CB3B47708370C670062229000430002DA1
:1067600011D004F0C5FE019B21006381029B0098BB
:10677000A381039BE381049B2382059BA37404F004
:106780001FFF07B0F0BD04F08BFEECE7F7B50093F8
:1067900008AB1B8807000C200D001600019304F0C5
:1067A0005FFE041E13D0280001F042FF00280FD026
:1067B0000078D0232370C93BA370009B2100238164
:1067C000019B6770A580E680638104F0F9FEF7BD48
:1067D000014B1878EDE7C0462045FF1F13B50400B4
:1067E00064890389C2888188C0780094FFF7CEFF4E
:1067F00013BD000010B5044C2068002803D004F03D
:10680000E7FF0023236010BDC066FF1FA122F0B583
:10681000818892004A43384B384F1B6804009B180C
:106820009D2292009B18827989B01A603B68002BE8
:106830005FD01D78324B1B68002B04D05B68002BA7
:1068400001D000209847260008363100E079FFF794
:10685000B7FD237DE0710200E0780493638A29008C
:106860000393238A0293E3890193A388009333005F
:10687000FFF752FFE378002B0BD1E289A379A188BF
:1068800002920196E27928000092012201F0DAFEDC
:10689000E0703B68002B20D0FFF7ACFF194D287843
:1068A00000281AD0184B1978FFF778FE002814D06A
:1068B0002B78E67808200793A78804F0D1FD011E05
:1068C00009D0D0230370CA3B4670837087808671DD
:1068D000079804F075FE00232B701721A088FFF79E
:1068E00075FCA08801F034FCA08801F00BFD09B014
:1068F000F0BD064B9DE7C0463409FF1FC066FF1F71
:10690000D466FF1FB566FF1FB466FF1F2045FF1F3B
:10691000F8B5070008000E0001F08AFE041E18D02A
:106920002620FFF78DFC051E00D12578062004F0F7
:1069300097FD041E0DD00021062204F0B1FDD023E6
:106940002370C23B21006770A370A680E8B204F0F8
:1069500037FEF8BDF0B585B001930AAB1B78070090
:1069600002930BAB1B7808000D000092039301F01B
:106970005FFE061E22D0102004F072FD041E1DD002
:106980001022002104F08CFD2620FFF759FC00287E
:1069900000D13078D0232370C13BA370009B21002D
:1069A0002372019B67706372029BA580A372039B95
:1069B000C0B2E3720C9BE36004F002FE05B0F0BDD0
:1069C000F7B50D00019001F033FE071E20D00E2018
:1069D00004F046FD041E1BD02620FFF731FC061EE6
:1069E00000D13E78D0232380C53B0622A370F91D39
:1069F000E01C04F07DFD019B2A0063810123DD4042
:106A00001A401D40210022736573F0B204F0D8FDD6
:106A1000F7BD0000F0B585B0029010000D00170022
:106A20000A9E039301F004FE041E31D0029B002B4A
:106A30002ED1039B02795B0724D512231343042232
:106A4000002E08D10B99002905D10C99002902D1FB
:106A50000D9900291AD01A430D9B2271002B00D0EA
:106A6000C9E0002E00D1CFE0002D00D0CCE0606A5C
:106A7000002801D004F0ACFE1C21300004F078FDA9
:106A8000606205E002239A430E33D7E793432371F4
:106A9000654BBA00D458002C00D1AAE0002E10D0CB
:106AA000236A002B03D11C2004F05AFD20625E4BA8
:106AB000BA00D358186A002803D01C22310004F011
:106AC00017FD0C9B002B12D0574CBB001D596B6A55
:106AD000002B03D1162004F043FD6862BB00E3588D
:106AE000586A002803D016220C9904F001FD0D9B72
:106AF000002B11D04C4DBC006659B36A002B03D15A
:106B0000142004F02DFDB0622B59986A002803D0A0
:106B100014220D9904F0ECFC380001F089FD051EEB
:106B200067D0414BBA00D358002B62D01A6A342088
:106B3000002A00D11C389A6A002A01D0143080B291
:106B40000B9A002A01D01C3080B25B6A002B01D066
:106B5000163080B204F084FC041E4AD018220021B2
:106B600004F09EFC2620FFF76BFB0190002801D16A
:106B70002B780193D0232370029B200063700A239B
:106B8000294EA370039BBD00A371AB59A780196A5E
:106B90001830002905D01C22A06004F0A9FC2000B8
:106BA00034307359996A002907D003001422143332
:106BB000E060029304F09CFC02980B9B002B08D031
:106BC00003001C221C330B992061029304F090FCFB
:106BD00002987359596A002903D01622606104F0A3
:106BE00087FC6B462100187904F0EAFC3800FFF7B7
:106BF000E3FC05B0F0BD10220D9B0D991B69A01898
:106C0000236204F075FC2CE70B9B002B00D13FE7BF
:106C1000012D00D03CE7606A002801D004F0D8FDC7
:106C20001C210B982AE7C046BC66FF1F10B5044C18
:106C30002068002803D004F0CBFD0023236010BDA2
:106C4000B066FF1F0B4B07B51A68002A01D1002060
:106C50000EBD6946531C012012780731FFF772FC04
:106C60000028F4D002780123100018401A42EED018
:106C7000EEE7C046CC66FF1FF0B51F4F01203B6812
:106C800087B0002B25D09B78059300F0B3FB00283C
:106C900021D00A20FFF7D4FA04000B20FFF7D0FA26
:106CA000164B05001E78731E9E413B68F6B2191DF7
:106CB000D878FFF757FB3B682900DA7A0433039250
:106CC0009A7901930292009033002000059A04F013
:106CD00047FE07B0F0BDFFF7B5FF002805D006203E
:106CE000FFF7AEFA04000720D8E70820FFF7A8FA5C
:106CF00004000920D2E7C046B066FF1FAC66FF1F44
:106D000070B50A4E040033780D00FF2B0DD004201F
:106D100004F0A6FB011E08D0D0230370CE3B4570C3
:106D20008370C470307804F04BFC70BD3045FF1F99
:106D300070B5040006200D0004F092FB011E0AD07D
:106D4000D0230370CD3B8370054B44701B68858056
:106D5000187804F035FC002C01D0FFF767FF70BDF8
:106D6000B066FF1FF8B5264F06003B680D001124E2
:106D7000002B05D10522234B1B78134202D112248C
:106D80002000F8BD204A10241268002AF8D012789A
:106D9000002AF5D0DB0719D52B789A1E012A1AD8BC
:106DA0000C2004F0DDFB132438600028E8D0002319
:106DB0000A22437029000670023004F099FBFFF7A5
:106DC0005BFF041E0AD0FFF731FFD9E700F012FB8A
:106DD0000028E1D1E4E7002BE2D0D0E70B4B1B7891
:106DE000032BCDD11D20FFF72BFA094B188000286B
:106DF000C6D0084B04211878074A04F001FBBFE70E
:106E0000B066FF1FAD66FF1FCC66FF1FAC66FF1F9D
:106E1000AA66FF1FD866FF1F60EA0000F7B501935E
:106E2000194B14001A78052306000F0012201A428D
:106E300021D0012920D1154B1D68002D1BD0022027
:106E40001F2C18D8002C02D0019B002B13D0104B04
:106E50001F221E706E1C0021300004F021FB0199DE
:106E60002200300004F044FB310020002C70002F81
:106E700006D004F075FAFEBD064B12201D68DCE753
:106E800004F0CEFBF7E7C046AD66FF1FCC66FF1FE0
:106E90003045FF1FC866FF1FF8B50F4E1224336838
:106EA000002B17D01B780F3C834213D100250B4FCA
:106EB0000221387804F034FA094B042138781D8017
:106EC00004F02EFA074B28001D8033685C7004F034
:106ED000FFFA04002000F8BDB066FF1FD866FF1F50
:106EE000C466FF1FAA66FF1F70B5012823D11B4C83
:106EF0002388002B03D01A4A1578002D07D0194B90
:106F00001B68002B02D01878FFF7C6FF70BD3B2B23
:106F100002D93C3B2380F9E7134E0221307804F07C
:106F2000FFF9FA222388920002215A43307804F0B4
:106F30002FFD2580EAE70B4B1B68002BE6D00B4B9F
:106F40001B785B07E2D5084B0221187804F0E8F9BA
:106F50000022024B1A80FFF769FED7E7C466FF1FC5
:106F6000A866FF1FB066FF1FD866FF1FAD66FF1F34
:106F7000F8B51E4D2868002803D004F029FC002332
:106F80002B601B4E3068002803D004F021FC002346
:106F90003360184F05243B7818002040234221D04D
:106FA000154800F02BFA3B78234213D0202004F040
:106FB000D7FA2860002813D02022002104F070FAAC
:106FC000202004F0CDFA041E306005D020220021DC
:106FD00004F066FA002004E0286804F0F9FB2C6055
:106FE0001320F8BD00F00AFAF4E7C046CC66FF1F94
:106FF000C866FF1FAD66FF1F2445FF1F10B50A4C72
:1070000023681A1E0ED0002808D10130587004F0F1
:107010005FFA002805D02368002B02D00021FFF77B
:1070200087FE0122100010BDB066FF1FF7B5274E86
:10703000050033680191181E21D05C78244F012C83
:1070400030D1FFF7FFFD002825D02000FFF7F8F82A
:107050000400412814D91F4B022118781E4A04F05D
:10706000CFF91E4B3C3C1C80022233685A703B789F
:10707000002B14D128000199FFF75AFE0120FEBD14
:10708000FA2292004243002AEED0124B02211878D5
:1070900004F07EFCE8E7FFF7D3F80200F3E70023F3
:1070A0003B70EBE73B78002BE8D1032004F0D8F9E4
:1070B000011E08D0D0230370CC3B45708370336829
:1070C000187804F07DFAFFF7B1FDD7E7B066FF1F2F
:1070D000A866FF1FD866FF1F60EA0000C466FF1F96
:1070E00010B51749838802008B4220D011D815496A
:1070F0008B4217D0144900205B1899B2012907D898
:10710000926811785A425341D8B2FFF7F9FD012035
:1071100010BD0E4A00209B1807229BB29A424041A4
:10712000C0B2F5E783681878FFF768FFF0E7836877
:1071300099785A78090218781143FFF777FFE7E743
:107140000A20000006200000F8DFFFFFAFDFFFFF8E
:10715000014B18707047C0463145FF1F10B5064CF3
:10716000207001F041FA207804F0CAF80521207857
:1071700000F062FD10BDC046D866FF1F0BB273B5AC
:107180000D00002B00DBC4E0884B187804F0E0FB16
:10719000041E0ED00378912B0FD0A22B00D1A1E0BA
:1071A000834B1878FF2852D0210004F009FA0028F8
:1071B0004DD180200002684076BD43780F2B76D0F9
:1071C00013D8052B70D00E2BEAD18088794B9842CA
:1071D0002BD8794B98421BD8784B9842E0D1A368C2
:1071E0001878591CFFF774F838E03E2BD8D1837813
:1071F000032B74D06CD8012B6ED0022BD0D1704BE6
:107200001B68002B23D05B68002B20D098471EE022
:107210006C4BC0180C28C3D804F0D2FA1DC2C2159A
:107220000BC20B0B0B3223C23C00674BC018072864
:10723000B6D8664B1B68002B09D01B68002B06D004
:10724000200098470AE0A3681878FFF7C7F82000E5
:1072500004F086FAADE7A068FFF762F800289FD037
:10726000F5E7A3681B78002BF1D0554B1B68002B6A
:10727000EDD01B68002BEAD0210055489847EDE778
:107280004F4B1B68002BE2D01B68002BDFD0210086
:107290005048F3E7504B1B68002BD8D05B68002B9D
:1072A000D5D021004348E9E7FFF7EAF9CFE7808826
:1072B0004A4B984203D04A4B984200D070E7464B65
:1072C0001B68002BC3D05B68002BC0D02100D5E722
:1072D000153B012BBBD963E7FFF798FAB7E7FFF738
:1072E0007DFAB4E73F4B1B78042B07D100236A4695
:1072F00013800179408800F0C5FCA8E7364B1B6875
:10730000002BA4D05B68002BA1D001003648984721
:107310009DE7012421420AD0294B1B68002B04D091
:107320005B68002B01D000209847012043E78B07C2
:107330000AD5264B1B68002B04D05B68002B01D0BC
:1073400020009847022036E70421280008400D421B
:1073500000D131E7254E3388002B21D0013B9BB271
:107360003380002B1AD1FFF7DBF800280AD0204B1E
:107370001C70164B1B68002B04D05B68002B01D0DF
:1073800020009847FFF7C6F8694601F001FD6846FE
:10739000FEF7FEFF1D20FEF753FF308004200AE7B2
:1073A000024B187803F0BCFFF8E7C046D866FF1F11
:1073B0003145FF1F0E2000000120000009100000D1
:1073C000D066FF1FFEDFFFFFAFDFFFFFD466FF1FAA
:1073D0000C2000000B200000B866FF1F0D200000ED
:1073E00013200000AD66FF1FFFFF0000AA66FF1F0D
:1073F000A866FF1F10B501F09BF910BD014B186086
:107400007047C046D466FF1F0B880020162B01D89A
:1074100017230420014A13807047C0468266FF1F6D
:1074200000207047074A03001188814207D09188E5
:107430000020994202D101308000101870470020CE
:10744000FAE7C046E066FF1FF0B58F7806000D0032
:10745000C7B01E2F15D1FFF7E5FF051E03D100248D
:10746000200047B0F0BD00223B003100C078009200
:1074700000F0B2FB0400A81C00F0D3FBFF23EB706C
:10748000EEE7264B062403931B78FF2BE8D0182F3A
:10749000E6D87B08224A013BDB0002929A589446C8
:1074A000002ADDD0029AD3185B68002BD8D0087868
:1074B000002802D14B78012B02D10624122FCFD104
:1074C00007AFAB88697800976446AA68A047041E96
:1074D000C6D1AB78029A5B08013BDB00D3183900B8
:1074E00030005B689847041E0BD1AB78042BB6D0F4
:1074F000039A310010782200009700F06DFB040021
:10750000AEE76A78002AABD1AA7805A93B88087152
:1075100030000A704B80FEF747FBA0E73445FF1FA1
:10752000ACBB00111D4B37B5050098420BD00029AC
:107530000AD1FFF777FF002805D11948FFF772FF3E
:10754000002800D0058037BD01291AD1FFF76AFF56
:10755000041EF8D001235B420380A378FF2BF2D0F6
:10756000FE2B07D00023E0781422009329001E335D
:1075700000F032FBA01C00F054FB01235B4263804F
:10758000E1E70229DFD1013901F0BEF80028DAD1A4
:107590002800FFF747FF041EDFD1D4E7FEFF0000FD
:1075A000FFFF0000022210B5074B52421A80074825
:1075B00001325A809A80DA8000F07EFA044801F0A5
:1075C00025F8002010BDC046E066FF1F4974001179
:1075D000257500110388F7B50400002B02D10225A0
:1075E0002800FEBD42680221137825485268FEF744
:1075F000A5FD00282ED0234F01253A88002AEFD080
:10760000802321885B0201259B1A9942E8DC0C202B
:1076100003F0A6FF061E31D03B8822889C4600233B
:107620001800019561469DB2491989B2AA421BD83A
:10763000002801D062443A8000233000082208C0AC
:10764000210003F055FF104A1368002B13D10025C9
:107650001660C5E76268022113780C485268FEF78D
:107660006DFD0028C7D1BAE760681D01401941814E
:1076700001330198D6E71A001B68E6E71325AFE748
:107680001ABC00113245FF1FDC66FF1F18BC001139
:10769000014B18707047C0463445FF1F14230A0081
:1076A00010B51A40194204D00122102101F048F807
:1076B00010BD4B06F9D4012088434000F8E710B50F
:1076C00014008B0604D50122102101F039F810BDF9
:1076D00008230A001A40194202D14BB2002B0FDADC
:1076E000102101F02DF8002808D02300F9331B7871
:1076F000002BECD0F8342378012BE8D10020E6E70A
:1077000003208907FAD4E2E7F0B51F00184B85B0D3
:107710001C68019002910392002C27D1200005B033
:10772000F0BDA5683301ED186B89019A934211D31E
:10773000029A93420ED8002F04D10A9B002B10D13D
:107740002C00EBE73B002978039A6868FEF7F6FC0B
:107750000028F2D10136B6B2A388B342E1D824683A
:10776000DAE7A3680A9A5B891380E9E70026F3E762
:10777000DC66FF1F37B50C000A8849880123914257
:1077800017D3002A15D0651D23792A0002210A4843
:10779000FEF7D4FC102300280BD0237961882088C1
:1077A00000242A000094FFF7AFFF0A23A04200D074
:1077B000230018003EBDC0461ABC001113B50A00D4
:1077C00008884988012388420BD8002809D0002462
:1077D000137905320094FFF797FF0A23A04200D0E7
:1077E0002300180016BD13B50A0008884988012334
:1077F00088420BD8002809D0002413790532009460
:10780000FFF782FF0A23A04200D02300180016BD14
:10781000F0B58BB003904A8808880E00012382429D
:1078200055D3002853D00023012704AC2370002235
:10783000718813000092FFF767FF051E3ED0207885
:10784000002835D12B78022B18D167706A89830004
:107850000130E31880005A8069680222201803F082
:1078600047FE23780133DBB22370042B19D93B0088
:107870006889013080B2002BD9D01FE002236370E9
:10788000122358436A89231804305A8069681022E9
:10789000201803F02DFE23780133DBB22370002B78
:1078A000E5D10C4A6B899B185A425341DBB2DFE7A2
:1078B0006378012BE4D12B78022BC7D022780A23DE
:1078C000002A04D021000398FEF798F9002318003D
:1078D0000BB0F0BD0100FFFF0F4BF0B504001868BE
:1078E000002816D083685D89A54207D88288AE1823
:1078F000B44203DA12019A18934201D10068EFE70B
:107900001E005F891036A74204D1002900D00D80E7
:107910001800F0BD3300EFE7DC66FF1F70B505000F
:107920000C0008880021FFF7D7FF03000120002B7F
:1079300004D022002800197AFFF7C1FE70BDF7B508
:107940000C00002501902300F6331B78AB4201D8D0
:1079500000200AE06B00E65A00213000E718FFF72C
:10796000BBFF002802D126800130FEBD017A0198BC
:10797000FFF794FE002802D03B882380F5E701350D
:10798000EDB2E0E710B5040008880021FFF7A4FF7E
:1079900003000120002B03D02000197AFFF77EFEA0
:1079A00010BD0000054B1B68002B01D1180004E03E
:1079B0009A6852898242F6D198887047DC66FF1F28
:1079C000F0B50E27002687B0039302ABFF183E8068
:1079D00005001F4B40891400984207D02B780130D6
:1079E00000976A6880B2FFF78FFE060002212B78AD
:1079F00018486A68FEF7A2FB00280FD06C892000A7
:107A0000FFF7D0FF002802D0013C0419A4B2039B69
:107A1000002B00D01C80300007B0F0BD02212B7875
:107A20000D486A68FEF78AFB0028E7D102212B780F
:107A30000A486A68FEF782FB002807D0002EDED0D5
:107A40003B88A342DBD17489013CDFE76C89DEE728
:107A5000FFFF00001ABC001118BC001116BC001179
:107A600010B50C00FFF7DEFC03000220002B0AD04B
:107A7000002C00D023609B781720FE2B03D0013808
:107A8000FF2B00D1002010BD73B50D0001A904002B
:107A90001600FFF7E5FF172805D0002E04D12900B6
:107AA0002000FEF727F976BD01221021200000F00A
:107AB00047FE0028F3D0F6E7014B18607047C04638
:107AC000EC66FF1F37B56B469D1D010004000222C6
:107AD000280003F07DFC2B88B02B0ED12379122BCC
:107AE00009D12300FF339B78012B06D10121608847
:107AF00000F0E0F801E01B2BF8D037BD10B5054BC6
:107B00000421187000F098F8FFF74CFDFEF770FBA9
:107B100010BDC046F066FF1F0020F0B50BB20F008D
:107B200087B0834234DA274B187803F011FF051E23
:107B30002BD00378A02B25D103AE3100FEF7E4F85B
:107B4000041E0BD1B378DB0724D51F4B06341B680A
:107B5000002B03D03100688898470400A8680028EB
:107B600001D003F015FC002C08D1184A039B1340E8
:107B7000174A934206D0B3781B2B03D001216888A3
:107B800000F098F8280003F0EBFD80200002784018
:107B900007B0F0BD0F4B1B68002B10D03100688878
:107BA0009847041EDAD07378002BD7D1B27801A998
:107BB0000A704B800C716888FDF7F6FFCEE706244B
:107BC000F1E7C046F066FF1FE866FF1F00FFFF00F9
:107BD00000011200EC66FF1FF7B501908220400003
:107BE0000D0017001E0003F03BFC04001320002CC6
:107BF00012D0B02320002370089BFC2267706580A0
:107C000026710830002B08D0190003F071FC210008
:107C1000019803F0D5FC0020FEBD089903F040FC5C
:107C2000F5E710B5041E06D00078FD2803D803F050
:107C3000A7FCFF23237010BD0A1F93B210B50400E8
:107C40000220032B05D882400020024BD1529B1802
:107C50009C7010BD1067FF1F0B8870B5043B0400BB
:107C60000D000220032B0BD80121200000F04CFD59
:107C700003001420002B03D02900200000F0DEFBBD
:107C800070BD000007B51300034A00920A000121ED
:107C900000F02CFC0EBDC046C17E001107B501925C
:107CA00003220092024B0A00122100F049FC0EBD93
:107CB0003F7F001107B56B4601AA11800449D880A7
:107CC00008780633012802D1190003F059FE07BDD8
:107CD000F166FF1F0C4B10B518700023FF210B4AF3
:107CE0001380138193819380094A538013705172DA
:107CF00093819372D174D3821375517703F050FE40
:107D000000F0FCF910BDC0462067FF1F1067FF1F81
:107D1000F266FF1FF0B58DB06B46002003910C2278
:107D20009B5E834200DBB0E05D4B187803F010FEF1
:107D3000051E00D1A4E00378902B00D09DE006AF93
:107D400001004688380000F013FA79680400002921
:107D500000D19CE03B88052B6ED13B89032B1CD9BD
:107D600005AC200000F0A2F86288172A61D8398992
:107D7000131D994231D17968237804310291D907D2
:107D800038D5607800F08EF9071E06D00023037105
:107D90002378012B08D0132B23D0A868002800D10A
:107DA00078E003F0F5FA75E06288029909A800F01E
:107DB000A6F80290380000F08BF909AA2378387AE7
:107DC0000192002231000092029A00F012F938006C
:107DD00000F064F9029B002BDFD0300000F080F946
:107DE000DBE70378032BD8D16288029909A800F059
:107DF000D6F8DEE7122B13D1029909A800F0B5F8E6
:107E0000021EEAD127498B88002BC6D0887909A9A0
:107E10002378019161780091310000F0EAF8BCE725
:107E2000002302AA93833000617809AAFFF72AFF92
:107E3000B3E71D4B0993F6E7042B02D09A1F012AE2
:107E4000ABD8184A043B9B00995A0029A5D0D218F8
:107E5000907831003A0000F0AEF800289DD13B88C0
:107E6000042B03D001213000FFF724FF012C04D1A3
:107E7000A868002801D003F08BFA280003F070FCFA
:107E80008020039B0002434018000DB0F0BD012884
:107E900000D182E701213000FFF70CFFEDE7C0467B
:107EA0002067FF1F1067FF1F010017000B7803708A
:107EB0004B784370CB788A781B021343438070471A
:107EC0000A88030002700A88120A42700A88012A8E
:107ED00006D14A8882704A88120AC270042070470C
:107EE00002208242FBD14A8804309A704A88120AE2
:107EF000DA708A881A718A88120A5A71EFE710B507
:107F00000400012082420CD94B780A781B021343EB
:107F10002380834206D1CB788A781B021343638087
:107F2000002010BD022BFBD1CB788A781B021343B3
:107F300063804B790A791B021343A380F0E70B8817
:107F400003700B881B0A43704B8883704B881B0A95
:107F5000C3708B8803718B881B0A4371CB88837134
:107F6000CB881B0AC3710820704703000120082A30
:107F700014D14A780878120202431A80CA788878A5
:107F8000120202435A804A790879120202439A8007
:107F9000CA798879120202430020DA80704710B54E
:107FA00004000120022A05D100204B780A781B0228
:107FB0001343238010BDF8B5060010200F001500F4
:107FC00003F04EFA04000120002C0ED0A0230C2256
:107FD000290023806780201D002D07D003F088FA38
:107FE0002100300003F0ECFA0020F8BD03F058FA4D
:107FF000F6E7F7B51E00009008AB142017001D78B7
:10800000019103F02DFA041E12D0A2230370019BEC
:1080100047704380099B057146710C220830002B84
:1080200007D0190003F064FA2100009803F0C8FAA1
:10803000F7BD099903F034FAF6E737B5041E0FD0FF
:108040004388002B0CD00025C1881323007A172207
:1080500001950095FFF7CDFFFF23658063722570C2
:1080600037BD000010B50C4904004A88002A09D029
:108070008B89002B05D00020CB8A0222834201D0BD
:1080800010BD012213000A20434300204032C8548F
:10809000C81842800472F3E7F266FF1F0023438092
:1080A00003707047094B00211A0010B55C88002C42
:1080B00006D01C79844203D10A234B43D01810BD4B
:1080C00001310A330329F1D10020F8E7F266FF1FDE
:1080D00010B50400407A03F053FAFF23637210BD19
:1080E0007047043010B580B203F0FAFA002803D0CC
:1080F0000421494203F05CFB10BD000070B500256F
:10810000104CA0682580A581A580A84202D003F06C
:108110003FF9A56000250C4C0C4B606D1D802300C1
:1081200058331D70A84202D003F032F9656500256E
:108130006068002801D003F02BF9013508340A2DBE
:10814000F6D170BDB867FF1F5C67FF1FAC67FF1FEC
:1081500070B5041E09D1054D2880A881A880A868A3
:10816000002802D003F014F9AC6070BDB867FF1F9F
:10817000F0B54B8885B00193002343600A79050070
:108180000F00022A00D07BE0CA88032A17D98B6827
:108190005E7819783602DC78D8790E4399781B7AA4
:1081A00024021B020C43034353495BBA0B80331D6B
:1081B00093421ED1042C04D0631F022B0ED9012040
:1081C00015E0019A4D4B1201D35A002B06D00198AD
:1081D000FFF7BEFF4A4A1369013313610421B868EF
:1081E0002E812C80494203F0E3FA6860002005B03C
:1081F000F0BD434D042C06D0631F022B0FD9EB6852
:108200000133EB60DBE7019A3C4B1201D35A002BA0
:1082100005D00198FFF79CFF2B6901332B61374B89
:1082200030000293019B029A1B01019300230199E4
:108230008C468B52130063449C8003939E81FFF70E
:1082400050FF039B041E986016D00421B868494271
:1082500003F0AEFAFA880100043A200003F048F96E
:108260000199029AFB888A5A043B9B18029A8B5206
:108270002B6801332B60A2E7AB690133AB619EE74A
:108280001E4B0293019B1E01029BF35A002B2DD023
:1082900002998C19A068002828D0012A26D1FA88D2
:1082A0009B189BB27352A189994217D39B1AC0188D
:1082B000B96803F01DF9029BA289F35A934200D0DA
:1082C0007DE700222B81A3882B80A3686B60029B33
:1082D000F2520B4A53680133536070E7084A9368BF
:1082E000013393600198FFF733FF68E7044A53694D
:1082F00001335361F6E7C0462267FF1FB867FF1FCF
:108300002867FF1F70B5051E15D10B4C0B4B18804D
:10831000230058331870606D002802D003F038F83D
:108320006565250050356068002801D003F030F8FD
:108330000834AC42F7D170BD5C67FF1FAC67FF1F0C
:10834000F0B51700A12285B0920001934243394B4A
:1083500006001B680C009B18D933FF331D78FDF70E
:1083600041FF0430854204DD3000FDF73BFF04305F
:10837000C5B2BD4207D33A0000213000019B03F093
:1083800067FA05B0F0BD2900380003F079F8230042
:10839000C6B250331E700393019B290063653800F9
:1083A00003F0A6FACBB20293002B02D0039B013656
:1083B0001E7000262300503303931B78B34204D869
:1083C000606D002831D10020DBE7029A2800002AE6
:1083D00004D0013B1000B34200D02800F700E71999
:1083E000387003F035F9786000280ED03A7801999A
:1083F00003F07EF8019A3B780136D3180E4A0193B8
:10840000D369F6B20133D361D4E7039B187060657A
:10841000A74205D1084A1320D36A0133D362B0E7DB
:10842000606802F0B5FF0834F2E702F0B1FF002304
:108430006365C8E73409FF1F2867FF1FF7B50D0004
:1084400007000421686803F0B3F92B890400037066
:108450002B891B0A43702B8883702B881B0AC370DF
:108460002E8902250436F6B2FB2E15D81B4B9F42EF
:1084700014D10C2002F0F4FF1135011E0CD0902312
:1084800003708E3B0371043B4380154B8460C680B0
:10849000187803F095F800252800FEBD5C237B4387
:1084A000104AD3180093583301931B78002B0FD137
:1084B0000300320038000099FFF742FF019B0500DE
:1084C0001B78002BE8D13800009903F0F9F8E3E7B6
:1084D000054A0725536A01335362DDE7FEFF0000BA
:1084E0002067FF1F5C67FF1F2867FF1FF0B587B07D
:1084F000009017200F0016000193FFF7F2FD1325DF
:10850000041E19D00C98031E02D00199201D984713
:10851000030AE370052302AAA0700430908127703B
:108520000098667003A993800494FFF787FF051EE7
:1085300002D0200002F02CFF280007B0F0BD0000A0
:10854000F0B587B01F000CAB1B7803910593012198
:108550000DAB06001C78049200F0D6F81425002814
:1085600021D02000FFF77EFD0135041E1BD01149EC
:10857000059B0A7803700132D2B2131EC68001D166
:1085800001231A000B7022713000049B039900979D
:10859000FFF7ACFF051E09D1230021000648074A5A
:1085A000093303F0EDF8280007B0F0BD0023638025
:1085B0002370F8E72467FF1F3B800011307500002F
:1085C000F8B505000E00064C064F2368002B02D0BC
:1085D0003100280098470434BC42F6D1F8BDC046AB
:1085E000C867FF1FDC67FF1F0123064A5B425380F9
:1085F000002313715362044A136053609360D36085
:1086000013617047DC67FF1FC867FF1F020000236C
:1086100010B506499C000859002801D1625010BDD0
:108620000133052BF6D11320F9E7C046C867FF1FB9
:10863000034A5388181A4342584140421040704739
:10864000DC67FF1FF0B585B002930AAB1F780CAB57
:108650001B88009008000E0001920393FFF7E8FFCB
:1086600005001120002D1BD10E48FFF7E1FF04008B
:108670001520002C14D006220B99A771E01D02F0E2
:1086800037FF019B30002371029B29006371009B1F
:1086900066802370039B6562E381FFF791FF2800EA
:1086A00005B0F0BDFFFF000010B5FFF7C1FF0400EB
:1086B0000220002C12D060880121FFF781FF606A40
:1086C000002801D003F084F828220021200002F0C5
:1086D000E7FE012300205B426380207110BD000093
:1086E00030B5074A074C5588010013780020A54291
:1086F00004D05B1A59424B415842104030BDC0462D
:10870000DC67FF1FFFFF0000084A10B501230C00C3
:10871000904208D0FFF78CFF031E04D0037923405A
:108720005A1E9341DBB2180010BDC046FEFF000088
:10873000024B1879431E9841C0B27047DC67FF1F97
:1087400070B504000D001600FFF772FF002804D179
:108750000D4B9C4200D0143070BD416A0379052056
:10876000002907D012221A40102A02D10520002E1B
:10877000F2D10F20DB06EFD5897E0C20A94289417A
:10878000494249420840E7E7FEFF0000030010B5F8
:10879000002800D110BD0348034A41889142F9D016
:1087A0009847F7E7DC67FF1FFFFF0000002330B5A5
:1087B000C45CCD5C6C40D4540133102BF8D130BD77
:1087C0000F23002210B5C45C64002243CA54C25C6B
:1087D000D209013BF7D210BD0200010010B52032D2
:1087E000103102F09DFF10BDF0B58BB0039010204A
:1087F00005931700049102F0B3FE0090102002F0E0
:10880000AFFE009B13240190002B05D000280CD153
:108810001324009802F0DCFF019B002B02D018000B
:1088200002F0D6FF20000BB0F0BD102002F098FE41
:108830000600102002F094FE13240500002E00D143
:10884000AEE0002819D01022002102F029FE3200EB
:108850002900039802F064FF041E0ED133787F2BA9
:1088600051D830000099FFF7ABFF009B1B787F2B9E
:1088700053D801990098FFF7A3FF300002F0A8FF3A
:10888000002D02D0280002F0A3FF002CC1D110203F
:1088900002F066FE0600102002F062FE0290002E3A
:1088A0007CD0002878D03A000F3223000125121125
:1088B00005D00F333B4015B25A4253411BB26A1EDA
:1088C0001201002B33D0049BD2B298180099029A5F
:1088D000FFF76CFF013D10220021300002F0E0FDA7
:1088E000ADB2049F2D017D19AF4242D0002C33D090
:1088F000300002F06DFF029B002B00D189E71800C9
:1089000002F066FF85E729003000FFF759FF2800D5
:108910002549009AFFF74AFFA7E729000098FFF7CB
:108920004FFF28002049019AFFF740FFA5E70F21DC
:108930000F4004998A18D9B28F4208D9D15C06A891
:1089400019540133102BF6D1029A0199C0E7791A14
:1089500048424141C901F2E73900300006AAFFF759
:1089600025FF3200039806A902F0DAFE1037040052
:10897000BAE7002CBCD13000029906AAFFF716FF17
:10898000320006A9039802F0CBFE08220400310051
:10899000059802F0ADFDABE71324A9E71324AAE77D
:1089A000002800D06EE733E720BC0011F0B58BB093
:1089B0000F0016000225009000283FD0002A3DD06D
:1089C0000B1DDBB21800029302F0CAFD1135041E24
:1089D00034D0FDF747FD05003A000099201D02F054
:1089E00097FFEBB20393E3702B0CDBB22F0A0093DB
:1089F0006370FFB22B0E2370A7700193FDF72CFD5F
:108A00001022010006A802F083FF2100029A04ABA5
:108A100006A8FFF7E9FE051E0DD1039B082233705F
:108A2000009B04A9B370019B7770F370301D02F0B6
:108A30006FFFFDF71DFD200002F0CAFE28000BB0FD
:108A4000F0BDF0B58FB00D00149E03900492059315
:108A5000002A03D1022420000FB0F0BD002EF9D06F
:108A60000398FFF7E5FD1424071EF4D072783378DD
:108A700012021A43B3781B041343F27812061A4306
:108A8000036A0192934201D30133E3D1002D03D055
:108A90003B7901249B07DED50822002106A802F0BD
:108AA000FFFC059B13240433DBB21800029302F091
:108AB00057FD051ECFD0059A0499043002F028FF17
:108AC00004223100280002F023FF39001022103167
:108AD0000AA802F01DFF2900029A06AB0AA8FFF7B8
:108AE00083FE041E0FD1082206A908A802F010FF79
:108AF0000822311D08A802F02BFD012807D1019999
:108B00000398FDF7C9FC280002F062FEA3E70124E8
:108B1000F9E7000070B51C4C05002368181E10D042
:108B2000002D14D11A78002A0CD1981C083202F0BA
:108B3000DFFC02F01DFE0135002808D123681D70FE
:108B4000012070BD0A331800082202F0D1FC23680E
:108B5000002BF5D0122002F083FC061E0DD0C1239D
:108B600021680370457002311022023002F0C0FC0F
:108B700023683100587802F023FD206802F028FEB7
:108B800000232360DCE7C0460468FF1FF8B504003B
:108B90002020FDF755FB0D4EA700BB590500002B0B
:108BA0000DD000280BD0D878FF2809D108492A0019
:108BB0000C55F35907480333611802F0E1FDF8BD85
:108BC000290002F02DFC0028F0D1F8E72068FF1FF3
:108BD0000868FF1FE59D001170B5064D84006359BC
:108BE000002B05D0D87802F0CBFCFF226359DA7055
:108BF00070BDC0462068FF1F70B506008CB00C0029
:108C0000150000213022684602F04AFC3100102293
:108C1000684602F07DFE1D2021000322684402F018
:108C200077FE6846FFF7D8FD2D21040003222800B7
:108C3000694402F06DFE20000CB070BDF0B5070075
:108C4000160097B001931CAB1D7830221EAB00912B
:108C50000AA800211C7802F023FC102239000AA87F
:108C600002F056FE1022002102A802F019FC072291
:108C7000310002A802F04CFE072202AB9818631ED6
:108C80009C41019902F044FE02AB9C732B005A1EDA
:108C9000934102AAD3730021102206A802F000FC1F
:108CA00006221D9907A802F033FE1A2002ABC01855
:108CB00006221F9902F02CFE102200990EA802F045
:108CC00027FE102202AB0EA908781C78013A6040FA
:108CD000D2B2087001330131002AF5D10AA8FFF79A
:108CE0007BFD102212A904000EA802F001FC102244
:108CF00006AB0EA908781D78013A6840D2B2087018
:108D000001330131002AF5D10AA8FFF765FD0443BC
:108D100010222098E4B212A902F0FAFD200017B048
:108D2000F0BD70B50E0014008CB001001022684632
:108D30001D0002F0EDFD3100082204A802F0E8FD5C
:108D40002100082206A802F0E3FD6846FFF744FD73
:108D500004001022280008A902F0DAFD20000CB05F
:108D600070BDF8B506000D0000243719AC4200D3E1
:108D7000F8BD02F08DFD030A3B70631CDBB20137C6
:108D80009D4203D90234F054E4B2EEE71C00EDE753
:108D900073B506000C000225002819D0002917D051
:108DA000032101A8FFF7DDFF6B469A793F231A40A4
:108DB000013313436A463000937101A92200FFF783
:108DC0001BFF051E04D10322E01C01A902F090FB49
:108DD000280076BD03785807DA08C00FD20080005B
:108DE0009B0710439B0F1843C0B2704707230B40EB
:108DF000C908C9000B4303707047000070B5040038
:108E0000FFF7EAFE134DA4006359002B21D0186A26
:108E1000002801D002F0DCFC2B59986E002801D00C
:108E200002F0D6FC2B59D86E002801D002F0D0FCFD
:108E30002B59186F002801D002F0CAFC2B59586F2B
:108E4000002801D002F0C4FC285902F0C1FC002324
:108E50002B5170BD2068FF1F0E4B8000C35870B5AA
:108E60000C00002B0FD09D68002D0CD02B78201DFE
:108E70000B706B784B70A97CFFF7B8FF2B7E2372C9
:108E80006B69E36070BD10220021200002F008FB36
:108E9000F8E7C0462068FF1F014B18607047C046C6
:108EA0001C68FF1F074A03008000825810B5002A83
:108EB00006D0D088984203D1012901D1FFF79EFF47
:108EC00010BDC0462068FF1FF0B5264E95B0870044
:108ED0000B93BB590500099112200A92002B31D047
:108EE000D888FFF7A5FB04001420002C2AD0280006
:108EF00010A9FFF7B1FFBB591E781D6A002E23D0C1
:108F00000895FDF7EFFA07000020FDF7F1FA07904A
:108F1000A379E61D069310AD0CA9089800F0E2FABB
:108F20000EA9280000F0D7FA0B9B0A990493069B20
:108F300009980293079B0396019300970EAB0CAA26
:108F4000FFF77CFE15B0F0BDFDF7CCFA06903000BF
:108F5000FDF7CEFAE31DA779079310AB060008933F
:108F6000DAE7C0462068FF1F30B50C4C85002A594F
:108F7000030085B00120002A0ED018006946FFF7D3
:108F80006BFF2B591A78D888054B002A00D1054B66
:108F90006A46072100F0D9FB05B030BD2068FF1FED
:108FA000D7940011E594001130B5094C850029597A
:108FB00085B010226846253102F09AFA2A5911210B
:108FC000044BD0886A4600F0C0FB05B030BDC046F7
:108FD0002068FF1F8195001130B5094C8500295983
:108FE00085B010226846353102F082FA2A591121E3
:108FF000044BD0886A4600F0A8FB05B030BDC046DF
:109000002068FF1FBF950011F7B54D4F8600102057
:10901000F4590D0002F0A4FAF3592062186A1322E1
:1090200000286CD0033A29009C6802F061FAF359D9
:109030001A780192002A58D11E6A227D317B94460B
:1090400051400122019F114201D167461740217D05
:10905000914339432175377B4F40BC46604600271A
:10906000800701D44F081740012102208F40227D44
:1090700082433A432275377B5740BC4660460027FF
:10908000400701D497080F400420227DBF0082438F
:109090003A432275627D002794466046727B4240C7
:1090A0000A4201D167460F400121627D8A433A435B
:1090B0006275777B5740BC4660460027800701D425
:1090C00057080F400220627D7F0082431743677577
:1090D000767B00227E40760701D4BA080A40042637
:1090E000617D9200B1430A4362756A78002A08D014
:1090F0006278002A05D005220533DA7700221000B5
:10910000FEBD04222979114205D1A17C114202D170
:109110000533033AF1E7019A21782C78002A02D12D
:109120000A002100140018220429E8D8042CE6D8EB
:1091300005206043034A05331218525CDDE7C04640
:109140002068FF1F30BC001110B50A001121024B2E
:1091500000F0FBFA10BDC0461B9600110B0030B5A5
:1091600087B001AD2B806B4604001100981D0822CA
:1091700002F0BEF92A000B212000024B00F0E5FAB4
:1091800007B030BD4396001110B50A001121024B03
:1091900000F0DBFA10BDC0469796001113B50B0026
:1091A00011006A4613706B4604000622581C02F038
:1091B0009FF96A4608212000014B00F0C6FA13BD52
:1091C000B796001110B50A001121024B00F0BDFA4C
:1091D00010BDC046079700117FB505000B4BAA00D4
:1091E000D4580800002C0FD0666F237FE2882178C6
:1091F0000396266F0296E66E0196A46E0094FDF724
:1092000009FC2800FFF7FAFD7FBDC0462068FF1F5C
:1092100010B51721FFF7E0FF10BD000070B50A0080
:109220000D00064B0221040000F08FFA0600297899
:109230002000FFF7D1FF300070BDC046E795001158
:1092400070B586B000236A461370836804001D78E9
:10925000681E0A2859D801A902F022FB06063337F6
:109260003B3F43474B4F5300180000F042F90623A1
:1092700012284BD000281BD16088FFF7D9F90823AA
:10928000002813D04279002A47D1264B1A780723A9
:1092900012070BD5244B1A680723002A06D016683C
:1092A000002E03D0290001AAB04703006A461370BC
:1092B0006B461B786088002B2AD1FFF767FC06B04D
:1092C00070BD180000F06CF9D4E7180000F087F9C1
:1092D000D0E7180000F093F9CCE7180000F0ADF9E2
:1092E000C8E7180000F0C3F9C4E7180000F0F6F969
:1092F000C0E7180000F0F6F9BCE7180000F013FA18
:10930000B8E7180000F013FAB4E707236A461370B1
:1093100069466088FFF782FFD1E70523012AC5D19E
:10932000024BB8E7AD66FF1F1868FF1F1C68FF1FE0
:10933000F8B52C4F8600F35904000D00002B40D0E7
:10934000DA8882423DD15A78062A33D11A78002A27
:109350002ED0012099681A6A097D014206D0157B3A
:10936000054203D007225A700120F8BD02200142B5
:1093700004D0157B054201D00922F4E70420014204
:1093800004D0127B024201D00B22ECE7164B1B6883
:10939000002BE9D05B68002BE6D020009847BB5932
:1093A00000215B78122BDFD12000FFF715FFDBE7F0
:1093B0000E4BECE7112A04D1002900D032252900F8
:1093C000F2E7002D08D12000FFF732F9002803D082
:1093D000102302791343037121002800FDF798FA46
:1093E000C2E7C0462068FF1F1868FF1F1C68FF1FE8
:1093F00070B50E4E8500AB590400002B13D01B78BE
:10940000002B11D10A4B1B68002B04D05B68002B8A
:1094100001D02000984773595B78122B03D10021AB
:109420002000FFF7D9FE70BD024BECE72068FF1F5C
:109430001C68FF1F1868FF1F094B8000C3581020CD
:10944000002B0CD01A6A002A09D09B68002B06D08A
:10945000127A1B7E101C9A4200D9181CC0B27047A9
:109460002068FF1F70B503000D0014000220002AC1
:1094700030D000292ED013700B78081D53704B7814
:109480009370FFF7A7FCE070012002212B7A237173
:109490006B7B034063716A7B0A4013430422637150
:1094A0006E7B1640334363716E7BF608F6003343E0
:1094B00063712B7B0340A371287B014000200B4389
:1094C000A371297B0A401343A3712A7BD208D200DF
:1094D0001343A37170BD10B50A0001000120FFF70E
:1094E000C1FF10BD10B50A0001000220FFF7BAFF4E
:1094F00010BD70B506000C000220002E30D00029EF
:109500002ED07378201D0B70B3784B70F178FFF775
:109510006DFC01223579257271794B1008001340DA
:10952000934010400343881010408000C908034353
:10953000C9000B436373B1794B100800134093408B
:1095400010400343881002409200C9081343C90029
:109550000B4321202373FCF773FE854201D21220B6
:1095600070BD2220257AFCF76BFE8542F7D8237860
:109570001820042BF4D86378012BF1D80020EFE7F2
:10958000030010B50220002909D0002B07D00322C8
:10959000481C0A7019000D3201F0AAFF002010BD0E
:1095A00003000222080010B5002B06D0002904D0C9
:1095B0000E32591C01F09CFF0022100010BD030068
:1095C00010B50220002909D0002B07D00422481C26
:1095D0000A7019000C3201F08BFF002010BD10B58D
:1095E000FFF7DEFF10BD03000220002906D0002B8C
:1095F00004D0052200200A701B784B7070470300CE
:109600000220002B08D0002906D05B7800200B70C8
:10961000013B082B00D918307047030010B5022019
:10962000002909D0002B07D00622481C0A70190017
:109630000A3201F05DFF002010BD10B5FFF7B0FF4A
:1096400010BD02000B00022010B500290ED0002A28
:109650000CD007211970118859701188090A997066
:1096600011180822D81C01F043FF002010BD030090
:109670000A00022010B5002B0CD000290AD09978DE
:109680005878090201431180901CD91C082201F06E
:109690002FFF002010BD030010B50220002909D0C3
:1096A000002B07D00822481C0A701900921801F0FC
:1096B0001FFF002010BD02000B00022010B5002982
:1096C0000BD0002A09D00921197011781818597087
:1096D000511C062201F00CFF002010BD10B5FFF751
:1096E0005FFF10BD02000B00022010B5002A09D058
:1096F000002907D05178197011180622581C01F062
:10970000F7FE002010BD030010B50220002909D08B
:10971000002B07D00A22481C0A701900063201F0FB
:10972000E7FE002010BD10B5FFF73AFF10BD0200A4
:109730000B00022010B5002A06D0002904D0180022
:109740005178FFF753FB002010BDF0B585B017002E
:109750001E006A4606230500080091819380FEF7EB
:10976000C0FC1324011E02900CD03800B047041E28
:1097700005D1280001A9FEF76FFA041E02D0029855
:1097800001F006FE2800FFF701FA200005B0F0BD49
:10979000F0B504008BB0019115000021102202A841
:1097A00001F07EFE334EA700B85900283CD0C38894
:1097B000A34239D10378002B36D14278062A18D13A
:1097C00002000100553235310C3006ABFFF7A9FA23
:1097D000002829D12000FFF72FFE020006A902A8C9
:1097E00001F086FE200002A902F09AF801200BB0D9
:1097F000F0BD816E002917D00B8A112A28D19D4215
:109800000ED101981231093A01F0A2FE012807D1C8
:10981000BB5920009D6EFFF70FFE29000200DEE716
:1098200032212000FFF7D8FC2000FEF701FF061EC2
:109830001BD0416A002918D00B8AAB4215D10822EF
:109840000198123101F084FE01280ED1716A0AE0FC
:109850009D42E9D108220198123101F079FE0128D8
:10986000E2D1BB59996E8A7EB9E7200002F080F8F8
:10987000BCE7C0462068FF1FF0B56B4D87007E59DE
:1098800085B0337802900393002B00D087E0B36853
:10989000346A01937078062817D101221B7D134288
:1098A00002D0217B114218D10222134202D0217B27
:1098B000114251D10422134203D0237B134200D022
:1098C0008BE0019B5A7DEB5991E007380428F8D8CA
:1098D00001F0E6FF032E42678300B36E002B03D135
:1098E0001C2001F03DFEB066EB599C6E002C1CD094
:1098F00010220021200001F0D3FD0298FFF79CFD0B
:1099000001002000FFF72DFA01F0C2FF20822000A5
:1099100008211230FFF725FA0298FFF78DFDA07697
:10992000EB592100D888FFF70FFC0822EB591CE007
:10993000B36E002B05D01A00198AF0881232FFF797
:109940000DFC0222019B197DEB5911423DD0207B79
:1099500010423AD0073208E0F488FCF7DBFD010042
:109960002000FFF711FC0A22EB595A70029B9C0061
:109970002A595378073B042B11D8D088FEF758FE9C
:1099800000284ED0C3895A08D2182849029B029851
:10999000CB542B5941180433254801F0F1FE05B092
:1099A000F0BDFCF79FFD03000120834201D10020A0
:1099B0000393EB59DE88FCF79BFD0399020030000E
:1099C000FFF7ECFB019AEB59117D042211420CD0F8
:1099D000217B114209D00B22C7E7F688FCF73CFD3A
:1099E00001003000FFF7EEFB6BE7019A527D012189
:1099F0000A4204D0607B084201D00C22B5E7022164
:109A00000A4204D0607B084201D00E22ADE7042157
:109A10000A4204D0627B0A4201D01022A5E712223A
:109A2000A3E7FA225200B0E72068FF1F2468FF1F57
:109A3000EF9D001110B5064B1A7804231000184052
:109A40001A4200D00348FFF727FA002010BDC04695
:109A5000AD66FF1F3845FF1F70B50400FFF7D4FA4D
:109A6000051E43D12000FFF77FFA234EA400A05922
:109A70008268937CDB0708D50321036A1B790B40BE
:109A8000012B02D1017F0B430377431DD97F8B1E2E
:109A9000022B0DD8022900D00121C088FCF790FFCD
:109AA000042133591A7F59700A431A77280070BD70
:109AB00001290CD102231022437000210C3001F047
:109AC000EFFC305910213530FFF74BF9EEE705294F
:109AD000ECD10223D118437010220C3001F008FDA4
:109AE00004233259117F0B431377EAE7082518281E
:109AF000DCD1053DDAE7C0462068FF1FF0B58BB02A
:109B0000059143887E4F9E00F45915000493002C64
:109B100015D1012902D000200BB0F0BD101D5778DF
:109B20001678FFF757F9EB68320002932B7A049905
:109B3000019300903B002000FCF70CFFEBE7E3886B
:109B4000049A934201D00820E6E72378012B00D144
:109B5000D4E0059B581E092800D9CFE001F0A0FEF3
:109B600005CE0A29CC506C859AB229000498FFF7DB
:109B700073FFD1E7200029001022453001F0B8FC26
:109B8000B9594B78042B02D1013B4B70C3E70B0052
:109B90000A00253335320C310498FFF795F9049803
:109BA000FFF702FA0522431E9841BB59C0005A70C4
:109BB000B2E7200029001022553001F099FC049BE7
:109BC0004F4C9D00295904980A0006AB55320C31C0
:109BD000FFF77AF929591022453106A801F0B8FC9F
:109BE000012808D10498FFF7F7F90590002804D15F
:109BF00006222B595A7005988EE708230593FAE739
:109C000063780C2B7AD1E36E002B03D11C2001F07A
:109C1000A7FCE066BB59D86E00286FD0102229003F
:109C200001F066FCBB590498DC6EFFF705FC0D22C1
:109C3000A076BB595A706EE7E06E00285ED063785C
:109C40000D2B5BD12B8808220382A91C123001F056
:109C50004FFCBB599A68517D0222114226D0186AE6
:109C6000407B104222D00C32E4E763780E2B45D1C2
:109C7000236F002B03D1162001F072FC2067BB5923
:109C8000186F002803D01022290001F031FC0F22A8
:109C9000BB59CFE763780F2B30D1206F0622691CA8
:109CA000103001F025FCBB599A68517D0422114205
:109CB00003D0196A497B1142D5D100210498FFF7DE
:109CC0008BFA28E7636F002B0DD0BB59586F002823
:109CD000F3D01022290001F00BFC0122BB595242A3
:109CE0005B6F1A61E9E7142001F03AFCBB59606729
:109CF0005B6F002BE9D126E72978DFE707200BE728
:109D00002068FF1F10B5064C207001F011FB0621E2
:109D10002078FDF791FF0348FEF778FC10BDC046A0
:109D20003368FF1FA58E001100200BB270B50D0027
:109D3000834216DA264B187801F00AFE041E0DD075
:109D40000378922B0ED0A02B37D0224B1878FF2807
:109D50003AD0210001F034FC002835D180200002E7
:109D6000684070BD43780E2B0BD03E2BEDD183782D
:109D7000052B12D0082BE8D181798088FFF7D8FA1B
:109D800008E0154B82889A42DFD183681878591C05
:109D9000FEF7C0FE002817D1D7E7104B1B785B07F2
:109DA00012D50F4B1B68002B0ED09B68002B0BD0DD
:109DB000C289811D80889847ECE7FFF741FAA068C7
:109DC000002801D001F0E4FA200001F0C9FCC5E749
:109DD0003368FF1F3145FF1F18200000AD66FF1FCD
:109DE0001C68FF1F10B50078FFF712FA10BD10B500
:109DF0000078FFF7FDFA10BD0C234343084A10B565
:109E00009B185A68002A03D0012901D1904710BD40
:109E10009B68002BFBD00029F9D19847F7E7C04693
:109E20005068FF1F01238340094A10B5946B1C43FF
:109E30009463506B98435063D46B2000984301297E
:109E400001D120001843D063116B0B43136310BD85
:109E500000800040F0B500240127154B85B0DA6B77
:109E6000144E03921A6C0192DA64019BE3403B4268
:109E700017D0039DE5403D400295E5B202992800C8
:109E8000FFF7BAFF316A736A002908D03900002B46
:109E900001D0029979402800FFF7C4FF01E0002BB0
:109EA000F9D101340C36172CDFD105B0F0BDC04616
:109EB000008000403468FF1F064B01215A68C240F1
:109EC0000A4204D01B68C3401800084070471B6D4D
:109ED000F9E7C046008000400122064B824000297D
:109EE00003D0D9680A43DA607047D9689143D960D2
:109EF000FAE7C0460038004030B5032444430F4B16
:109F0000E25C1B199C785D7801232D1B0135AB4069
:109F1000013BA340A140DB430C00122807D80849AD
:109F200092005218116819402143116030BD054A52
:109F300011680B4023431360F8E7C04677BC00115B
:109F400008F0004014F00040C21F70B5D4B20623E0
:109F5000092C0BD80125084C9540002908D0002178
:109F6000FFF7CAFF23682B4323600023180070BD4E
:109F70002368AB43F8E7C04600380040214BF0B5FA
:109F80001B185B78022B21D1032444431E4A1F4E29
:109F9000A35C12199478012215008540B76B013C2F
:109FA000E4B23D43A240B563194C122815D89B007A
:109FB00000290CD117495B1899680A439A6001235C
:109FC000205C154A834011680B431360F0BD1149B2
:109FD0005B18996891439960F1E70E4B00290DD108
:109FE00059690A435A61225C1328E8D00123203AB8
:109FF00093400A49086803430B60E7E759699143B6
:10A000005961F0E73468FF1F77BC00110080004001
:10A01000BCBC001100F00040A0F00040A4F00040E3
:10A02000F8B500241B4E1C4D1C4B1B5D012B1FD192
:10A03000194A9269E2401A420BD00122B25693406B
:10A040002200143AD2B2022A09D815494A691343A8
:10A050004B61013402360C35172CE5D1F8BD0022D6
:10A06000B2560F499200521891680B439360F0E783
:10A07000022BEED1E7B23800FFF71EFF0123584054
:10A08000C1B23800FFF77AFF3800FFF715FF687795
:10A09000DFE7C04649BC00113468FF1F3568FF1F69
:10A0A00000F00040012202388240054B002903D015
:10A0B00059690A435A617047596991435961FAE7EE
:10A0C00000380040F8B50E0001210F008740114A0A
:10A0D0000400D368FD43BB43D360831E8B4201D889
:10A0E000FFF7E0FF00212000FFF72EFF0A4A0B4B8D
:10A0F0005168012E05D139431B1951605E70002053
:10A10000F8BD2940516002221C1962709A691540FD
:10A110009D61F4E700380040008000403468FF1F74
:10A12000012210B58240074B002906D019680A4366
:10A130001A600121FFF7C6FF10BD1968914319602D
:10A14000F7E7C046008000400C2370B5002543436C
:10A150000A4A29009B181D70094B04001B185D70EA
:10A16000FFF7B0FF0123A340064928000A681A43FD
:10A170000A6005490A689A430A6070BD5068FF1F6B
:10A180003468FF1F348000403080004070B5040008
:10A190000E00FF2813D003250540FFF7D5FF084A1E
:10A1A000A3089B009B183F22ED00AA40AE4019680F
:10A1B00020009143314319600121FFF78DFE70BDEE
:10A1C00018380040F8B50C244443134B0500E4183C
:10A1D0006368002B03D1A3681220002B1AD002223F
:10A1E00001270E4B00215B195A7028002770FFF7DA
:10A1F00069FF63681E1E08D0A3683E00002B04D0D0
:10A200002800FFF759FE4640F6B228003100FFF75C
:10A2100009FE0020F8BDC0465068FF1F3468FF1FCC
:10A22000F7B5C420FF222B4B80001958002491431E
:10A230003F3A0A431A508022274F5202274E1A6093
:10A24000274B1D5D002D21D0A31E012B03D801211A
:10A25000E0B2FFF727FF012D18D11F4B9B69E340A8
:10A260002B4213D0E3B218000193FFF725FE010043
:10A270000198FFF755FFE3B2143B022B1DD80121D3
:10A280007156184A8D405369AB4353613B7F002B95
:10A290000DD0E5B22800FFF795FF2800FFF70CFE70
:10A2A0007B7F0100834202D02800FFF7A5FD013427
:10A2B0000C370236172CC3D1F7BD0121002371568C
:10A2C000F3568D40074A9B009B189A68AA439A60F0
:10A2D000DCE7C04600E100E03468FF1F49BC001124
:10A2E0003568FF1F00F0004010B501210400FFF7A2
:10A2F000E9FE0123044A002011194B70A340916923
:10A300000B43936110BDC0463468FF1F70B50E004B
:10A3100015000400FFF718FF0C236343094A2000CF
:10A320009B189D605E60FFF74DFFF021064B074ACA
:10A330008900051E5A5002D02000FFF705FF2800B3
:10A3400070BDC0465068FF1F0000FF1F559E0011E2
:10A3500070B5134D07202C78002C1FD198222100B6
:10A360005200280001F064FA0123C420FF222B7060
:10A370000C4B80001C635C630B4B1C605C600B4BE4
:10A38000195891433F3A0A431A50802252021A60E8
:10A390000D20074A074901F0A3FA200070BDC0460E
:10A3A0003468FF1F00800040A0F0004000E100E0A2
:10A3B00021A2001121A00011030010B50620072BD7
:10A3C00009D8054A137000F0EBFFD7210020034B9A
:10A3D000034A89005A5010BD6045FF1F0000FF1F4F
:10A3E000151BFF1F70B51D0002240C2910D8094A47
:10A3F000CA40D2070CD5FBF72FFF041E08D1059ADF
:10A4000004992800FBF744FFFCF7B2FDFFF712FBAD
:10A41000200070BD1210000030B50D7802232C0012
:10A420009C43184201D02B431C0008252300AB435A
:10A43000284201D02B00234320241D00A5432042A5
:10A4400001D01C4325002A230D70184204D0117836
:10A450001E3B0B43137030BD0028FCD10C21137838
:10A460008B43F7E7F8B51D0006AB1B88140007AA5D
:10A470000E000B201778002B27D10A78022A49D129
:10A480004A68507811780002244A0843801804284A
:10A4900040D801F005FA03121D1B2300F06801F0FB
:10A4A000B7F9021CC0B2B84200D93A1CD2B220009F
:10A4B000F1682A8001F01CF806E00222F3681B888C
:10A4C0002A8023701B0A63700020F8BD0622EEE785
:10A4D00001232B80F3681B782370F5E7F368002BCA
:10A4E00016D008222A801A8822701A88120A6270EE
:10A4F0005A88A2705A88120AE2709A8822719A8841
:10A50000120A6271DA88A271DB881B0AE371DBE749
:10A510002B80D9E701202B80D7E7C04600D6FFFF6C
:10A52000F7B516000A781D0008AB1F880C00012340
:10A53000022A18D14A685078117800022B4A084341
:10A54000801803280FD801F0ABF902254439E068E0
:10A5500001F05EF9C0B20723B84204D37B1901931E
:10A56000152B02DD0D231800FEBDE0682A00310026
:10A57000C01900F0BDFF6B4600209B88E268D054F4
:10A580001B4B1B68834203D01B68834200D0984753
:10A590000023E8E70B23002FE5D1022DE2D17378E9
:10A5A00032781B021343E2681380114B1B68002BA7
:10A5B000EED01B68002BEBD00120E8E70B23002F27
:10A5C000D1D1062DCED12A003100E06800F090FFF5
:10A5D000DEE70B23002FC6D1012DC3D132787533AE
:10A5E000012AC0D8E3681A70D2E7C04600D6FFFF40
:10A5F000406AFF1F70B50C001500072837D801F01E
:10A600004FF9041436361B36242E182015290BD882
:10A61000184E16220021300000F042FF22002900CF
:10A62000300000F065FF002070BD18200229FBD12A
:10A630001288114B1A80F6E718200829F4D10A0075
:10A640000E48290000F0C4FEEDE718200129EBD1E7
:10A650000B4B10780B49DA69FFF7DEFEE3E71820B1
:10A660000129E1D1064B10780749DA6BF4E70220A3
:10A67000DAE7C046286AFF1FDE45FF1FD445FF1FEB
:10A680006445FF1F8C45FF1FAC45FF1F030010B53D
:10A690000020DB0704D50721024A034800F08CF8AC
:10A6A00010BDC046D4BC00116445FF1F054A03001D
:10A6B0001068002803D082889A4201D180687047D0
:10A6C0000068F6E7446CFF1F0A88030008009A42FE
:10A6D00004D08A8804309A4200D0002070470000DD
:10A6E000F8B5F82200230D4F0D4E7968050042435E
:10A6F0003370994200D07B600A4C0021200000F0AA
:10A70000CFFE00231A007C60AB4202D100203370E0
:10A71000F8BD01332280DBB2F834F5E7446DFF1F4A
:10A72000406DFF1F486CFF1F73B56B46019006001C
:10A73000684615001980FCF74DFF041E11D1002D4D
:10A740000FD07689002E11D00C2000F009FF0028D0
:10A750000ED0084A0460136886808560002B02D101
:10A760001060200076BD1A001B68F7E70224F8E7A6
:10A770001324F6E7446CFF1F012100220A4B10B599
:10A7800049420A4C198099809A719A70084B20703E
:10A79000012019805A60FFF7A3FF2078FCF778FFAB
:10A7A0000448FDF733FF10BD486AFF1F4C6DFF1FC3
:10A7B000446DFF1F65A80011022310B5002802D0C8
:10A7C000FFF7B2FF0300180010BD0000030010B532
:10A7D0000020DB0704D50421024A0348FFF7A4FF49
:10A7E00010BDC046E8BC0011E445FF1FF0B50E26C1
:10A7F00087B003930CAB1F8802ABF6180500080066
:10A8000031000292FDF768F804000120002C0FD0FF
:10A810003088FFF74BFF03000E20002B08D05E6846
:10A82000002E05D021002800039B029A0097B04714
:10A8300007B0F0BD0A4B10B5984207D101220023A2
:10A8400052420A808B708A808B7110BDFFF73CFFEB
:10A850000028FAD001235B42038000238370F4E7D1
:10A86000FFFF0000F8B5050001290AD1134E0024AE
:10A870003388F827AB4219D028001149FFF7DAFFD7
:10A8800006E0022904D10139FDF73EFF0028EDD092
:10A89000F8BD3B0063437268D018D35A002B09D02F
:10A8A0003A00002100F0FCFD0134E4B2054B1B78B6
:10A8B000A342EED801235B423380DDE7446DFF1FE6
:10A8C000486AFF1F406DFF1F10B5FFF7FDFE030034
:10A8D0000020834200D0987810BD0000F0B589B008
:10A8E0001C000EAB80CB03901E8810AB1B7804922B
:10A8F00002930B7A0D00DB0616D42B780593022BFE
:10A9000024D00498FFF7D2FE002812D003689C469A
:10A91000002B0ED0029B2200019329003B006446CD
:10A9200003980096A04705E00498FFF7BFFE0028B3
:10A9300002D10E2009B0F0BD8368002BF9D00A22A5
:10A940002900039898470028D7D0F3E76B68587818
:10A950001A786B4B000210439842D2D8043B9842BD
:10A9600010D2684B984242D015D8674BC0180128C6
:10A97000C7D80B20002EDDD1EB681A7859683A80D1
:10A98000200028E0614BC018032800D979E000F0CE
:10A9900087FF846A789E5E4B9842B2D10B20002ECE
:10A9A000C8D101233B80EB6831001B782370688994
:10A9B000013080B2FCF790FF3A88031E0ED0017878
:10A9C00002328A183A80428962704289120AA27061
:10A9D00059680278E01C00F08BFD06E004323A80F2
:10A9E00031000422601C00F05BFD0020A2E70B2078
:10A9F000002E9FD1EB6807A91E8804233B80330AF1
:10AA0000300026706370FCF767FF051E28D004AB8A
:10AA10009A890E2304A95B183E49C668FCF7D0FF4B
:10AA200000280BD12B783C486A680599FBF786FB18
:10AA3000002803D1012304AA5B42D3813278022A81
:10AA400006D17168201D00F053FD3B8802333B8026
:10AA50000E2304AA9B181B88A3701B0AE370C4E78B
:10AA600004ABDE81F4E70B20002E00D062E7E9683A
:10AA70000398FFF729FF02233B802070000A6070D3
:10AA8000B3E70B20002E00D054E70222EB681B88AE
:10AA90003A8023701B0A6370A7E7E86800F0B8FEED
:10AAA000C2B203000720B24200D243E70DD00299A0
:10AAB000DBB27118994202DB921BD3B20293029B64
:10AAC000E9681A003B8089195AE70023F6E70B2052
:10AAD000002E00D02EE70722EB683A801A78227009
:10AAE0005A7862705A88A2705A88120AE2701A79EB
:10AAF0002271DA886271DB881B0AA37175E7C04690
:10AB0000042900000228000000D8FFFFFFD6FFFF45
:10AB100003280000FFFF000018BC0011F0B58DB045
:10AB20006B460020089120229B5E83423DDAA64BB3
:10AB3000187800F00DFF071E32D00378B02B2CD10F
:10AB40000079023816281FD800F052FD17001E00A9
:10AB50001E001E0031001E0096001E001D011E007A
:10AB600052011E0073011E00CD011E0050021E0086
:10AB70001E001E008E021E00E302944B94491B88A7
:10AB800078880B80FBF71AF83800FCF79BFF914B95
:10AB90001B68002B01D038009847380000F0E0FD1A
:10ABA0008020089B0002434018000DB0F0BDF62243
:10ABB0000021874800F074FC0BAA3B7B7989388917
:10ABC00000923A000D32FCF79FFD0400804B1B7889
:10ABD000002C3FD146E0804B788805937F4B4100A5
:10ABE000CB5A0BAE073BDBB23288029300230193B2
:10ABF0007B4B210006930093059BFFF76FFE744D7E
:10AC0000002810D1069B3A8A1B889A420BD1380043
:10AC10000599123000F09CFC002804D02B78628942
:10AC20009B00EB185A80162306A81B1832882000B8
:10AC30007989FCF7C5FE2B7804009A00AA18518880
:10AC40000029C3D00133DBB22B70002807D006A93E
:10AC5000C98A9180634A12889A42BCD802E00121D5
:10AC600049429180002B04D059497888FAF7DAFFDD
:10AC70008AE73E890A2479E000253E89574B0693EE
:10AC80007B88069A5B009B5A033B9D4202DB002DAA
:10AC9000F0D05BE0162206A812183B7B798900925F
:10ACA0003A0030000D32FCF72FFD0590002858D0F7
:10ACB0004689017A7888FCF7F1FC041E44D1464BA2
:10ACC00078880793069B4100C95A454B0439C9B29D
:10ACD00006AAD28A06930291019400930599079BD4
:10ACE000FFF7FCFD041E2FD1069B39491A88931CDF
:10ACF000002D26D14B807988384B4900CB5A511909
:10AD0000033B8B4220DD059B31485B8941190B7168
:10AD1000A91C0135C9B2EDB2059145191B0A2B7169
:10AD2000059B2D490433181800F0E2FB2C4B059AC3
:10AD30001B88D318DDB22C4B9E4205D00136B6B22B
:10AD40009CE749889942D6D0002D0CD0204C280091
:10AD5000618800F0D5FB207021007888FAF772FF37
:10AD600012E7059CF0E7002C00D183E77B78142BD9
:10AD700000D109E716493B794E800B700C71788839
:10AD8000FAF712FF00E7162406ABE4182100388911
:10AD9000FCF7A2FD011E00D1B7E1788822880F4C94
:10ADA00045002C5B0A4D013CE4B2029400240F4B99
:10ADB00001940095FFF792FD041E00D014E12900D4
:10ADC0007888FAF74FFFDFE64C6DFF1FD044FF1F76
:10ADD000506AFF1F446AFF1F4A6BFF1F8066FF1FF8
:10ADE000406CFF1FCE44FF1FFFFF0000526AFF1F91
:10ADF000162406ABE41821003889FCF76DFD011E0E
:10AE000000D182E178882288AE4C45002C5BAE4DA3
:10AE1000013CE4B202947C89AC4B01940095FFF7AD
:10AE20005DFD041E00D0DFE029007888FAF724FFDA
:10AE3000AAE60025A44B1D803B00FE331B78A24AE6
:10AE400078880792AB4208D99E4B128806930699E0
:10AE500043005B5A013B9A4203DB0799FAF716FF5E
:10AE600092E616246B00FB18059306ABE418059BCD
:10AE700021001889FCF730FD011E03D1059B012438
:10AE80001E8973E77888924B2288069C09934300B9
:10AE90001B5B904E013BDBB20293002300960193B3
:10AEA000099BFFF71BFD041E02D0059B1E895DE771
:10AEB0007B88069A5B009B5A079A10883288121882
:10AEC000934202DC1B1A013B33807F4C02303288F4
:10AED0000999001900F00CFB2388328801359B1872
:10AEE0002380EDB2A8E70BAA3B7B798938890092D1
:10AEF0003A000D32FCF708FC00250590059B002B5D
:10AF000004D10A24002D00D16EE060E0059B788812
:10AF1000197AFCF7C3FB0100041E63D1694C6C4B2A
:10AF2000788806940993069B4400E45A694B063CD2
:10AF3000E4B20BAE32880793029401910093059915
:10AF4000099BFFF7CBFC041E4CD1079B5E491B8875
:10AF50001A1D002D30D14A80059B5B4C5A8963191C
:10AF60001A716B1C9BB2E318120A1A71162306A8F9
:10AF700032881B1879890598FCF722FDFF21AA1C4D
:10AF80002E1D03350B00059092B2B6B2ADB200286B
:10AF900003D006ABDB8AD9B21B0AA218651911715E
:10AFA0002B714C4D301D2A884949201800F0A0FA19
:10AFB0002B88F618B5B2A1E74988914207D17A8863
:10AFC00006995200525AEB18053A9A42C4DC3E4C9C
:10AFD0002800618800F054FA207021007888FAF780
:10AFE0005FFED1E5002DF2D13E89BFE6162606AB05
:10AFF000F61831003889FCF76FFC3D000400FF357E
:10B0000000282DD0037A9B060CD400227B89398935
:10B01000788800923A000C32FFF7E8FB041E10D04B
:10B020003E8915E03088FFF741FB00281AD083687D
:10B03000002B17D02100122278889847041EE4D0F4
:10B04000EEE7AB78002B02D17888FAF739FE0026BC
:10B05000AB78002B00D097E5002C00D194E585E675
:10B060000124DDE70E24DBE7162506ABED182900E9
:10B070003889FCF731FC041E47D0037A9B0611D4B3
:10B08000154A7B881188994203D01448814207D120
:10B090001380134BF8261D780023D9B2A94221D37F
:10B0A0000924A1E72888FFF701FB00282FD0836837
:10B0B000002B2CD02100122278889847041EDFD064
:10B0C00092E7C0468066FF1F506AFF1F526AFF1F4B
:10B0D0004A6BFF1F406CFF1F446DFF1FFFFF000006
:10B0E000406DFF1F31005943546801336018615AA5
:10B0F0000029D2D13C0008342100F82200F0F8F9F0
:10B1000021007888FAF7E4FD3EE501246CE70E247F
:10B110006AE71D4B1A887B889A4231D07888FAF703
:10B12000E1FD31E5F823059851684343CD18C95A2C
:10B1300000291FD03B7A012B0BD16C88AB88788813
:10B14000AA1D0094FFF752FB041E02D000233B729D
:10B150002E88F8220021280000F0A2F900232B807D
:10B16000059B0133DBB20593084B05991B78064A12
:10B170008B42D7D801235B421380002CCED0F5E55B
:10B18000002634000596EFE7446DFF1F406DFF1F5A
:10B1900070B504000E001500FFF796FA031E08D1E3
:10B1A00031000548FFF790FA03001120002B02D070
:10B1B0001C8000209D7070BDFFFF0000F8B50B4F94
:10B1C00006003B780D001400FF2B0ED00A2000F083
:10B1D00047F9011E09D0B123038000234680037183
:10B1E000C5800481387800F0EBF9F8BD2546FF1FD3
:10B1F000F7B50F0008A90600088809A90B240988DB
:10B20000002821D10234022B1ED1557813782D024B
:10B210001D432B008B4301937334002B14D1FB6827
:10B22000300019000093FFF74FFB019C85420BD0C3
:10B230002A0030000099FFF7ABFF041E04D12A005A
:10B2400030007989FFF7BAFF2000FEBDF0B50E7817
:10B2500085B003900AA805880120022E0DD14C6804
:10B260002778647824023C43054FBC4205D10398FB
:10B27000DBB201960095FFF7BBFF05B0F0BDC046FD
:10B280000229000010B504000C4800F081FA0C48B7
:10B29000A16B00F07DFA0B48E16B00F079FA0A48E7
:10B2A000216C00F075FA094B0948196800F070FA32
:10B2B000084B1B68002B00D09847FEE7EABA001144
:10B2C00000BB00110FBB00111EBB001104ED00E01C
:10B2D0002DBB0011506DFF1F002307B501A801937E
:10B2E000FFF7D0FF044A0548002110B5121A00F0FC
:10B2F000D7F8F8F75FFBFEE7546DFF1F2846FF1FE6
:10B3000001B40248844601BC604700BF5D170000DD
:10B3100001B40248844601BC604700BF9DA90000FB
:10B3200001B40248844601BC604700BFB35201002B
:10B3300001B40248844601BC604700BFC926000032
:10B3400001B40248844601BC604700BF053AFF1FB4
:10B3500001B40248844601BC604700BF512500008B
:10B3600001B40248844601BC604700BF4D1F000085
:10B3700001B40248844601BC604700BFB14E0000E2
:10B3800001B40248844601BC604700BFC9A900005F
:10B3900001B40248844601BC604700BFD94901009E
:10B3A00001B40248844601BC604700BF151BFF1F63
:10B3B00001B40248844601BC604700BFB134FF1F9E
:10B3C00001B40248844601BC604700BFADAE000036
:10B3D00001B40248844601BC604700BF810E0000F2
:10B3E00001B40248844601BC604700BF35550000E7
:10B3F00001B40248844601BC604700BF456B0100B0
:10B4000001B40248844601BC604700BF59520100A4
:10B4100001B40248844601BC604700BF9538FF1F55
:10B4200001B40248844601BC604700BF5147010097
:10B4300001B40248844601BC604700BF4939FF1F80
:10B4400001B40248844601BC604700BF8552010038
:10B4500001B40248844601BC604700BFC56D0100CD
:10B4600001B40248844601BC604700BF1D4D010085
:10B4700001B40248844601BC604700BF3D1800008B
:10B4800001B40248844601BC604700BF090E0000B9
:10B4900001B40248844601BC604700BF5135FF1F1C
:10B4A00001B40248844601BC604700BF154D01004D
:10B4B00001B40248844601BC604700BF056A000031
:10B4C00001B40248844601BC604700BF913AFF1FA7
:10B4D00001B40248844601BC604700BF691F0000F8
:10B4E00001B40248844601BC604700BFC94A01005C
:10B4F00001B40248844601BC604700BFE94C01002A
:10B5000001B40248844601BC604700BF350E00000C
:10B5100001B40248844601BC604700BF01890000B5
:10B5200001B40248844601BC604700BF156B0100AE
:10B5300001B40248844601BC604700BF455000008A
:10B5400001B40248844601BC604700BFC537FF1FF5
:10B5500001B40248844601BC604700BFCD4C0100E5
:10B5600001B40248844601BC604700BF3D4B010066
:10B5700001B40248844601BC604700BFF94C010099
:10B5800001B40248844601BC604700BF1147010076
:10B5900001B40248844601BC604700BF3D3BFF1F29
:10B5A00001B40248844601BC604700BF4136FF1F1A
:10B5B00001B40248844601BC604700BFD13AFF1F76
:10B5C00001B40248844601BC604700BF594F0100E6
:10B5D00001B40248844601BC604700BFF30E00007E
:10B5E00001B40248844601BC604700BFB54C01006D
:10B5F00001B40248844601BC604700BF093DFF1FFB
:10B6000001B40248844601BC604700BFD1A50000D8
:10B6100001B40248844601BC604700BF055E0000DB
:10B6200001B40248844601BC604700BF55220000B7
:10B6300001B40248844601BC604700BF6571010047
:10B6400001B40248844601BC604700BFB93BFF1FFC
:10B6500001B40248844601BC604700BF017F00007E
:10B6600001B40248844601BC604700BFA137FF1FF8
:10B6700001B40248844601BC604700BFE530FF1FAB
:10B6800001B40248844601BC604700BFDD6601008A
:10B6900001B40248844601BC604700BFA54F0100C9
:10B6A00001B40248844601BC604700BF1D4B010045
:10B6B00001B40248844601BC604700BF8932FF1FC5
:10B6C00001B40248844601BC604700BF7D18FF1FDB
:10B6D00001B40248844601BC604700BF2146010016
:10B6E00001B40248844601BC604700BFE92800005D
:10B6F00001B40248844601BC604700BF2526000013
:10B7000001B40248844601BC604700BF2124000008
:10B7100001B40248844601BC604700BF6DBC000014
:10B7200001B40248844601BC604700BFE548000000
:10B7300001B40248844601BC604700BFEDA500008B
:10B7400001B40248844601BC604700BF8D1200006E
:10B7500001B40248844601BC604700BFC95C0100D7
:10B7600001B40248844601BC604700BF434D01005C
:10B7700001B40248844601BC604700BFD91B0000E9
:10B7800001B40248844601BC604700BFA9460100DD
:10B7900001B40248844601BC604700BFE53A01009D
:10B7A00001B40248844601BC604700BFF134FF1F6A
:10B7B00001B40248844601BC604700BF55490100FE
:10B7C00001B40248844601BC604700BFE13CFF1F52
:10B7D00001B40248844601BC604700BF014C01002F
:10B7E00001B40248844601BC604700BF75A900004F
:10B7F00001B40248844601BC604700BF9930FF1F76
:10B8000001B40248844601BC604700BF513AFF1FA3
:10B8100001B40248844601BC604700BFDD5201000C
:10B8200001B40248844601BC604700BF291C0000E7
:10B8300001B40248844601BC604700BFB70E000057
:10B8400001B40248844601BC604700BFC51D00002A
:10B8500001B40248844601BC604700BF5118FF1F75
:10B8600001B40248844601BC604700BFE53BFF1FAE
:10B8700001B40248844601BC604700BF7132FF1F1B
:10B8800001B40248844601BC604700BFC5210000E6
:10B8900001B40248844601BC604700BF2951010041
:10B8A00001B40248844601BC604700BFF53CFF1F5D
:10B8B00001B40248844601BC604700BF0124000077
:10B8C00001B40248844601BC604700BF0D5201002C
:10B8D00001B40248844601BC604700BFC53F000078
:10B8E00001B40248844601BC604700BF1133FF1F0A
:10B8F00001B40248844601BC604700BF090E000045
:10B9000001B40248844601BC604700BF193AFF1FDA
:10B9100001B40248844601BC604700BF45510100A4
:10B9200001B40248844601BC604700BF311B0000DF
:10B9300001B40248844601BC604700BFED4A0100E3
:10B9400001B40248844601BC604700BFC932FF1FF2
:10B9500001B40248844601BC604700BFF54E0100B7
:10B9600001B40248844601BC604700BF851F000047
:10B9700001B40248844601BC604700BF091B0000B7
:10B9800001B40248844601BC604700BFE1170000D3
:10B9900001B40248844601BC604700BF8B520100DD
:10B9A00001B40248844601BC604700BF791800001A
:10B9B0000002010302030303040305020602070257
:10B9C000080209000A030B030C020D000E030F030B
:10B9D000100311031303140315001600993D001101
:10B9E000CD3D00110000000002000000F2B900117E
:10B9F000192A0F180A000000F1590000FD24000068
:10BA000041460100157D0011299D00117D71001135
:10BA1000197B0011255300111DAB0011994F001126
:10BA2000913F0011C14000110000000016160000F7
:10BA3000020000003CBA0011F4FFF3FFD2FC00004A
:10BA400001420011000000000000000054757961FF
:10BA50000042312E32003030303100676974687531
:10BA6000622E636F6D2F70767678004254483031C5
:10BA7000000000000200000088BA0011292A282ACC
:10BA8000272A262A252A242A0A180000E204000070
:10BA90007102000078EC00007440000010270000E4
:10BAA00060F0000006640000204E0000000000006E
:10BAB000010000001F501D00023CB40000011400F2
:10BAC0001200000081020000303132333435363745
:10BAD0003839414243444546005048592B36325884
:10BAE00058504C555330353034005B4861726420F7
:10BAF0006661756C742068616E646C65725D0A00C5
:10BB00004C522020203D203078253038780A0050D3
:10BB1000432020203D203078253038780A005053CB
:10BB20005220203D203078253038780A0049435390
:10BB300052203D203078253038780A0029570011EE
:10BB40007D570011000000000200000054BB0011EE
:10BB50006F2A6E2A1A18000001A0000000000000E1
:10BB60006410B71DC8206E3BAC30D9269041DC76FE
:10BB7000F4516B6B5861B24D3C7105502083B8EDA8
:10BB800044930FF0E8A3D6D68CB361CBB0C2649BCC
:10BB9000D4D2D38678E20AA01CF2BDBDFB349B5FF1
:10BBA0008000008000100000000000007F5D001198
:10BBB00009740011A35D001111780011275E0011B6
:10BBC000E77700119D5E0011BD770011EF5E001157
:10BBD00085790011575F001185790011895F001187
:10BBE0003F7900119D5E001175770011155F0011FE
:10BBF0001D7900110000000000000000FB5F001133
:10BC00001D7900115D60001121740011052A042ABC
:10BC1000012A002A022903280128002801180018F7
:10BC2000000000000000000000000000000000878D
:10BC300001010201020101020102030304010301E7
:10BC4000010101010303020103000D000E001000B9
:10BC5000110013001401070108010A010B011C0166
:10BC60001D02040205020702080219021A021C0240
:10BC70001D03010302031700020100050400080769
:10BC8000000B0A001716001D1C010201010504012A
:10BC90000E0D011110011413011716011A190202D9
:10BCA00001020B0A020E0D021110021413021716E4
:10BCB000030504030807030B0A030E0D000102032A
:10BCC00007090A0B0E0F101112141718191A1B1F4F
:10BCD0002021220065A4001121A500110000000010
:10BCE000020000001EBC0011000000004DB2001157
:0CBCF00000000000020000001CBC00115D
:020000041FFFDC
:1000000000000000F53E0011F8B90011F4B900112C
:100010003463FF1F0000000000000000000000002B
:1000200000000000000000000000000000000000D0
:1000300000000000000000000000000000000000C0
:1000400000000000000000000000000000000000B0
:1000500000000000000000000000000000000000A0
:100060000000000000000000000000000000000090
:100070000000000000000000000000000000000080
:100080000000000000000000000000000000000070
:100090000000000000000000000000000000000060
:1000A0000000000000000000000000000000000050
:1000B0000000000000000000000000000000000040
:1000C0000000000000000000000000000000000030
:1000D0000000000000000000000000000000000020
:1000E0000000000000000000000000000000000010
:1000F0000000000000000000000000000000000000
:1001000000000000000000000000000000000000EF
:1001100000000000000000000000000000000000DF
:1001200000000000000000000000000000000000CF
:1001300000000000000000000000000000000000BF
:1001400000000000000000000000000000000000AF
:10015000000000000000000000000000000000009F
:10016000000000000000000000000000000000008F
:10017000000000000000000000000000000000007F
:10018000000000000000000000000000000000006F
:100190001535FF1F5D33FF1FC16601000000000021
:1001A000000000000000000000000000000000004F
:1001B000000000000000000000000000000000003F
:1001C000000000000000000000000000000000002F
:1001D000000000000000000000000000000000001F
:1001E000000000000000000000000000000000000F
:1001F00000000000000000000000000000000000FF
:1002000000000000000000000000000000000000EE
:1002100000000000000000000000000000000000DE
:1002200000000000000000000000000000000000CE
:1002300000000000000000000000000000000000BE
:1002400000000000000000000000000000000000AE
:10025000000000000000000000000000000000009E
:10026000000000000000000000000000000000008E
:10027000000000000000000000000000000000007E
:10028000000000000000000000000000000000006E
:10029000000000000000000000000000000000005E
:1002A000000000000000000000000000000000004E
:1002B000000000000000000000000000000000003E
:1002C000000000000000000000000000000000002E
:1002D000000000000000000000000000000000001E
:1002E000000000000000000000000000000000000E
:1002F00000000000000000000000000000000000FE
:1003000000000000000000000000000000000000ED
:1003100000000000000000000000000000000000DD
:1003200000000000000000000000000000000000CD
:1003300000000000000000000000000000000000BD
:1003400000000000000000000000000000000000AD
:10035000000000000000000000000000000000009D
:10036000000000000000000000000000000000008D
:10037000D9B20011000000000000000000000000E1
:10038000000000000000000000000000000000006D
:10039000000000000000000000000000000000005D
:1003A000000000000000000000000000951AFF1F80
:1003B000000000000000000000000000000000003D
:1003C000000000000000000000000000000000002D
:1003D000000000000000000000000000000000001D
:1003E000000000000000000000000000000000000D
:1003F00000000000000000000000000000000000FD
:081838006071FF1F4118FF1F42
:10184000024981F3088802F02BFC00006071FF1F41
:1018500010B502F02DFB072804D0122808D002286A
:1018600008D010BD044A0420136B01331363F8E75A
:101870000220F6E71420F4E72867FF1FF8B50700F9
:101880000C0026002500503630785135002804D150
:101890000300287058342370F8BD2978CA00481E08
:1018A0008141A3183800A25C5B68C9B2FFF7D0FF82
:1018B00000280DD12B78DA00A218013350602B706C
:1018C0003378044A013B3370136A01331362D8E75B
:1018D0000123DFE72867FF1F5C234343074910B557
:1018E000C9180B0058331B78012B05D1FFF7C6FF31
:1018F000034A936A0133936210BDC0465C67FF1FC1
:101900002867FF1F10B502F023FC064A01211300CF
:1019100010CB4942D967044B136002F059FC2000F8
:1019200010BDC04600E100E01000100010B504003A
:1019300002F00EFC024B1C6002F04AFC10BDC046D7
:1019400000E100E010B5040002F002FC4021094A69
:10195000200013688B43136002F052FB01F0BCFDC2
:101960000022054B01201A60044B04321A6002F079
:10197000D7FAFEE71CF00040C4F00040C0F0004081
:10198000431E5A425341A022F0B5D2015B4213409C
:10199000154D164A40019B182A18127E8BB00191F2
:1019A000002A1BD01A000832D46F0022E6B206AF1C
:1019B000E4B294420EDC2818C369002B08D00199C8
:1019C00002AA117106AA049202AA167303A89847E4
:1019D0000BB0F0BD1978B9540132EAE71A7D1A78D4
:1019E00006AB01261A70E6E7E869FF1F00400040D9
:1019F000F0B5254B04004001C25C85B0002A2BD015
:101A00001A18117E002927D0917E002924D011793F
:101A1000022921D11689D788D168F51BADB22A1CBD
:101A2000102D00D9102292B2BE4217D118180123EE
:101A300003710023C269C38003819A4206D06846BD
:101A4000032103730171029301A890470820002C21
:101A500000D0192001F038FC05B0F0BD013C654212
:101A60006C41A0256442ED012C40084D1B186419FF
:101A7000074D0633013A92B2AA42EDD01888461CAF
:101A80001E80085C2070F5E7E869FF1F00400040F9
:101A9000FFFF00000F220E4B10B59868104002386F
:101AA0000A280BD802F026F90D0A0B0A0A110A0AB5
:101AB0000A0A060002210020FFF762FF10BD012183
:101AC000F9E70020FFF794FFF8E7DB6FF6E7C04681
:101AD000004000400F220E4B10B5986810400238AD
:101AE0000A280BD802F006F90E0A0B0A0A120A0A93
:101AF0000A0A060002210120FFF742FF10BD012162
:101B00000800F9E70120FFF773FFF7E7DB6FF5E760
:101B10000090004013B5334C2378072B3DD8324B4F
:101B20001A78324B002A39D18022196852020A43AE
:101B30001A60252001F08CFF20232D4A11680B43E9
:101B4000802113606B460422C905086807331042E0
:101B500028D080210422C905C86810422ED08021D7
:101B60002020C905CA688243CA6014221A701A78F4
:101B7000002A2FD18021C905C86820320243CA60DB
:101B800014221A701A78002A28D11A4B1A7D22784A
:101B90005A601D221A705932DA6013BD1A6816494C
:101BA0000A40C5E7086802430A6014221A701A78CE
:101BB000002ACED01A78013AD2B2F7E7C8680243B9
:101BC000CA6014221A7019784A1ED2B21A700029FB
:101BD000F9D1C4E71A78013AD2B2C7E71A78013AC4
:101BE000D2B2CEE76045FF1F2846FF1F3CF0004001
:101BF0005845FF1F00200040FFFFFEFF564B70B509
:101C00001B68012B03D1554A936D0133936502F094
:101C1000B7F8534B534A1860534B544C1A60012386
:101C2000534A1360534A13602378002B06D00622D0
:101C30005149524802F00CFA00232370504A514B8C
:101C400010681B78C1B2002B0ED14F4CC0B2237864
:101C50005BB2002B4FDB237824785BB264B21B04A9
:101C600024021B191B1813600B1C50294ED950233A
:101C7000464A47491078DBB2FF2202284BD1086858
:101C8000444C454D267890432A78964254D9227880
:101C900024782E78023B5D10A31B6B435201D31AAC
:101CA00010335B111843086002F0EAF8031F012BA0
:101CB00045D83A4B1B78002B06D0394B1B78002BAC
:101CC00002D0002002F054FAA122364B92009978FB
:101CD000354B4A431B689B18832292009B181B7844
:101CE000033B012B03D8AF20400002F031F9012261
:101CF0002E4BDA8270BD237824785BB264B2FF3356
:101D0000FF341B0424021B190138ABE7CAB2022AB4
:101D1000AED20223ACE70868254C264D26789043C6
:101D20002A78964208D9227824782D78023B5B10D5
:101D3000641B63435201B2E72378DBB2B2E70228A7
:101D4000D5D11D4B1B78013B022B03D91B4B1B78B4
:101D5000022BCCD16C20C8E79809FF1FFC0FFF1F96
:101D60006066FF1FFF3F0000141003406466FF1F02
:101D70000C10034000100340D50BFF1F7211FF1F12
:101D8000B40003408C09FF1F680AFF1F490AFF1FA8
:101D900094000340460AFF1F470AFF1FF908FF1F70
:101DA0002209FF1F300DFF1F3409FF1FBC0BFF1F4F
:101DB000440AFF1F450AFF1F1C09FF1F2309FF1FBD
:101DC00010B502F085F80022014B1A8010BDC04604
:101DD0005C66FF1F10B502F043F9A121054A890096
:101DE0009478054A61431268044B5218528C1A8049
:101DF00010BDC046300DFF1F3409FF1F5C66FF1F7A
:101E000010B50D4B0D4A9978A1239B004B431268E6
:101E1000D218531DD97F0A4B1B88994209D2441C02
:101E200007D0C82805D0D2695B1A5A43054B5343E3
:101E3000C01802F0BDF810BD300DFF1F3409FF1FA0
:101E40005C66FF1F7102000070B5244D2B68002BEB
:101E500028D001F0A5FF2B68D8402B680400002B88
:101E600027D002F02DF82B68D8401D4B1D4A9978D9
:101E7000A1239B004B431268D118D25C91239B0095
:101E8000002A20D0CA580132CA50174B17491B6884
:101E90000868834214D3D23B181A012A1AD0144B73
:101EA000186070BD01F07CFF124B196802F088F8D1
:101EB000D3E702F005F80F4B196802F081F8D4E778
:101EC0000D495B18E8E7CA500C4B1B68DB68E41847
:101ED000201AE4E7F530FF30E1E7C0461C08FF1F99
:101EE000300DFF1F3409FF1F9C09FF1F6066FF1F95
:101EF000A009FF1F1808FF1F2DFF3F006866FF1F86
:101F000070B504000D00282916D10300A433C2883F
:101F10001B889B1A0B4A9BB293420DD906006A3666
:101F200005223100653002F03BF8002804D1310071
:101F3000200001F01DFF70BD2900200002F0A0F874
:101F4000F9E7C046FE7F0000F8B50400012001F06B
:101F50008FFF01F0F5FE194A03001060184E194872
:101F6000016831600568A942FAD11748174E056823
:101F700077680020AF4201D27068281A144D091901
:101F800028601448C162A421446A49032143416284
:101F900011490978002905D010490978022902D190
:101FA0000F3B1360F8BD012901D1083BF9E7032974
:101FB00001D1053BF5E7033BF3E7C046E408FF1F0B
:101FC000340AFF1F28F00040180AFF1F28100040A5
:101FD0001C0AFF1F00F000401C09FF1F4A0AFF1FD8
:101FE00070B580241025E405A3682B43A36001F09D
:101FF000CFFEA368AB43A36070BD0000F7B5160029
:1020000080221C001023D2050191916805000B432A
:10201000936000225A4BD7301A6001F0D1FE9D2305
:102020002A002F009B00EB58CA3201210092FC3796
:10203000002B01D00021009A386802F019F829001D
:10204000009BCB311A784F4BD3351A604B780A7806
:102050001B0213438A7812041A43CB781B061343DE
:10206000494A1BBA13604B790A791B0213438A79D8
:1020700012041A43CB7931001B061343434A1BBA9F
:1020800013606B782A781B021343AA7812041A4350
:10209000EB781B0613433E4A1BBA1360019A3302C6
:1020A00013433C4A13603C4B22001B1B9C460329F4
:1020B0003DDCB3089A0013005142B21A032A46D1FC
:1020C000354AE018511A827840781204000202431F
:1020D000E05C043302430A600022FF2B4BDDF02258
:1020E0002E4B12011A600F222D4B1A602D4A1368D5
:1020F000002BFCD00023224A27491360091B321D04
:102100000B191B68043A180A23706070180C1B0E18
:10211000A070E3700434002AF2DC802210213B68B6
:10212000D20501333B6093688B439360F7BD6346F0
:10213000D578981893782D061B042B43157804390D
:102140002B43557804322D022B430360AFE7022A5C
:102150000AD1114AE05C511AE21852781202024385
:102160000A6004339BB2B7E7012AB5D10A4A521A72
:10217000E15C1160F5E7084959180A600433ACE7DF
:10218000000004403C000440380004403400044097
:10219000300004400C0004400001044004000440EE
:1021A0001000044014000440F7B5150080221C0004
:1021B0001023D2050091916807000B439360002320
:1021C000654AD730136001F0FBFD9D233E009B0064
:1021D000F9583B00CA363200FC33002900D07FE0BA
:1021E000586801F045FF390032785C4BCB311A60FA
:1021F0004B780A781B0213438A78AC4612041A43C0
:10220000CB78281D1B061343554A1BBA13604B7924
:102210000A791B0213438A7912041A43CB791B06ED
:102220001343504A1BBA13604B7A0A7A1B021343BA
:102230008A7A12041A43CB7A21001B0613434A4AB6
:102240001BBA1360009A2B021343484A1360220002
:10225000474B1B1B0093009BCE785B1801938B7838
:1022600036061B0433430E78043833434E7804316A
:1022700036023343019E33600328ECDC0321A808B7
:10228000431C9B002940800003292BD13849E518C5
:102290005E18A9786D78E35C09042D02294319437F
:1022A0003160030008330021FF2B2DDD314B324913
:1022B00019600F21314B1960012327490B60304B06
:1022C00019680029FCD006211B680B40042B20D084
:1022D00080220020D20593680A318B439360FEBDB3
:1022E00001217DE7022908D121495D18E1184978CB
:1022F000E35C090219432960D3E70129D3D11C49C2
:102300005918E35C0B60CCE71948181801600433D6
:10231000CAE7002310490B606346002B0CDC3B002E
:10232000FC335A68102101325A608022D20593682A
:1023300001208B439360D2E7009B9B181B68190A0E
:1023400013705170190C1B0ED37004235B429170F3
:102350009C440432E0E7C046000004403C000440D6
:102360003800044034000440300004400C000440B5
:102370000001044004000440080F00001000044065
:102380001400044070B5061E19D00222614B9B79DF
:102390009343012B13D1604B1A78FF2A0FD15A783F
:1023A000FF2A0CD19A78FF2A09D1DA78FF2A06D1C0
:1023B0001A79FF2A03D15B79FF2B00D1A7E0574B95
:1023C0000C201A78012A08D00022554D1A702B785B
:1023D0001A00093A042A01D8212070BD5A1F012A87
:1023E000FAD94C4CA07B042800D990E0A279032AAA
:1023F00000D98CE0821E012A03D862881F2A00D8E7
:1024000085E0002E61D0012E00D080E0A288012A54
:10241000E2D0002B0AD10138032803D801F06AFC6E
:10242000151D19151F202E7001F08AFD2B785A1EDC
:10243000032A16D800253B4B1D602823237501F085
:1024400047FEA8422ED0A580C6E7022320202B708D
:10245000EAE7042322202B70E6E7032321202B70D8
:10246000E2E7073B012BB7D82F4B1B68DB6A9B06C3
:10247000B2D52E4B1A78002AAED1A27B911E01292B
:1024800001D9002AA8D1022280211A702823284DC0
:1024900089012878237501F033FE8021287889018D
:1024A00001F03EFC0123A380224B1B78002B0AD0B5
:1024B000FA228021204B92001B8809025A431C4BB0
:1024C000187801F055FD002087E701F041FE2B78D8
:1024D000A680073B012B06D918482E7001F0B0FEEC
:1024E0001E2001F02DFD114B114C1A78002A06D048
:1024F00080210022207889011A7001F001FE01F08C
:1025000067FE80212078090201F0FAFDDBE7122046
:1025100063E7C046A60BFF1F6B09FF1F1A09FF1FC9
:102520001C09FF1F4809FF1F6866FF1F2309FF1FC3
:102530001B09FF1F2109FF1F2C09FF1F001000406E
:1025400010B5002901D001F06BFC10BDF7B5604B50
:1025500001919978A1239B004B435E4A06001468C1
:102560001022E418D6235B00E0583623FF33E35CE7
:1025700000279343222B41D1574B0F3A1A60076033
:10258000012501F06DFE019B1880E8235B00E35CF0
:10259000002B01D0B34258DD0023504FFB70AD3308
:1025A000FF33E3581A68002A03D09B88DB439B075C
:1025B0001DD03823FF33E35C002B18D09B235B0036
:1025C000E35C002B13D1D133FF33E35CB3420EDA6B
:1025D000A4235B00E15AE018090A023101F058FC1B
:1025E00023000122FE33013E01351A87FA70E823E9
:1025F0005B00E35C002B2AD0A8B2FEBD03683D005F
:10260000002BBED081880430090A023101F040FC61
:10261000D6235B00E3581F60B2E72300B133BA0052
:10262000FF339858013781880430090A023101F0DC
:102630002FFCE8235B00E35CBB42EEDCE822F61AE9
:10264000ED1800235200A354A6E70027F1E720006D
:1026500001F056FC00281FD0002E1DDD73198826BE
:1026600047190193B600200001F0CAFB5A308000E0
:1026700020184068013581880430090A023101F0D0
:1026800007FC200001F014FDA3590133A351BD4202
:1026900002D0019B9D42E6D1114BE35C002BABD0F5
:1026A00095239B00E35C002BA6D00E4BE15A00293A
:1026B000A2D00D4AA35C994202D90133A3549BE7EF
:1026C00000231A212000A35401F092FD94E7C04694
:1026D000300DFF1F3409FF1F00140340E010FF1FDF
:1026E0005A020000720200005E020000F8B51D4BA5
:1026F0001D4F1A78002A10D1BA7B002A02D101326C
:102700001A7003E0032AFAD0022AF8D001F0E0FCA4
:1027100000220120154B1A70F8BD154B154D1C6891
:10272000154B9E7801232B702878C0B200F0DEFC98
:10273000BB7B002B0BD101F053FBA1239B00734308
:10274000E41883239B00E41823782B70E4E7032B21
:1027500002D101F06DFCF0E70020022BDCD101F08A
:10276000D7FBEAE71C09FF1FA60BFF1F2309FF1F6A
:102770003409FF1F490AFF1F300DFF1FF0B587B056
:102780000EAD2F780FAD2D780593AC46634614003F
:102790000E4D0CAA12782E7803930D9B0092019394
:1027A0002200059B029701F0FBFC2E70012C01D04A
:1027B000042C08D1802206498B889343054A12785D
:1027C000D20113438B8007B0F0BDC0461C09FF1F28
:1027D0006C11FF1F7809FF1F0B001B3B70B5040035
:1027E0003020E02B0DD81300E025493BFF3B9BB286
:1027F000ED00AB4205D8034B200019825A8201F04C
:102800001FFB70BD8410FF1F10B501F0B9FA054B16
:1028100000205B68052B04D9034A5268D20200D419
:10282000980810BD00100040FCE100E070B501F018
:102830008FFC0D4B1B68FC33DC691D6AFFF7E4FF5E
:102840006419844204D2094B01241B68002B07D071
:1028500004220024064B1A70064A936901339361DF
:1028600001F0B6FC200070BD6866FF1F9809FF1FCD
:102870002309FF1FFC0FFF1F70B50C4D2B68FC33A5
:102880005C6A01F065FCFFF7BFFF2B680025FC3395
:102890009B6AE318834204D2054B1B68AB4200D10C
:1028A000051B01F095FC280070BDC0466866FF1F3F
:1028B0009809FF1FD722044B92009B5810B5002B9C
:1028C00000D0984710BDC0460000FF1FF0B587B08C
:1028D00001F09AF9FFF7EEFFCA4BCB4C04931B783B
:1028E000022B45D1C94B1B68186A01F0C1FAC84BCD
:1028F000C84A1A60C84BC94A1A60A022C84B520085
:102900001A60049B187801F053FCC649C64801F0D0
:102910008FFAC649C64801F08BFA1022C54BFF203A
:102920001A60802252031A60802292031A60802269
:1029300012041A6001F01CFC012001F001FCFA20D5
:10294000400001F0F5F9582001F002FBBA4801F00F
:1029500017FB012001F004FB072001F069FC22684D
:10296000B64B1A4084235B001343236007B0F0BDCD
:1029700001F096FAB24E0290322001F079FA3368F3
:102980001B0629D43C2001F073FA0F2001F070FAE5
:102990009C4B1B78012B00D11EE180223368A94D8E
:1029A000134200D0A7E02B68032013432B6001F0F3
:1029B0005FFA01F075FA029B0299C31A5A1E81420E
:1029C00000D81A00A04B1A60904B19681E2353437D
:1029D0009E4A9B18CB618AE701F062FA80239C4AE9
:1029E000DB02116803900B4313602268934B994FED
:1029F0001A40282313432360032001F039FA0320EF
:102A00003D6801F035FA3B680320DB03DB0B0093E4
:102A100001F02EFA3B68ED03DB03ED0BDB0B8E4A76
:102A20000193AB18C22B30D8009B9B18C22B2CD81B
:102A3000019B9B18C22B28D8009B2A009D4200D2E4
:102A40001A00009B9D4200D91D00019B934200D2B9
:102A50001300019A954200D915005B1B122B14D864
:102A60000C22336814209343336033687B4A13404D
:102A7000336001F0FDF908213B682268DB038A43DB
:102A80002260774ADB0B13607FE7032001F0F0F947
:102A90003B68DB03DB0B059301F002FA039B039910
:102AA000C21A531E814200D813006E4A93421BD9AA
:102AB000FF23356869492D0A1D4032686B1C1B06CF
:102AC0000A401B0C134333600C23326800209A43E6
:102AD000083B1343336001F00BFA6348634BA84093
:102AE000984206DCFEF72EFF019B009D0093059B9C
:102AF00095E75F48F6E700235E4F554A3B60802329
:102B00001168DB020B43136080222B680320134300
:102B10002B6001F0ADF93B68052601333B60802353
:102B20002A685B0213432B602268444B03201A403F
:102B3000514B1343236001F09BF90821454B1A6860
:102B40002368D2038B432360454B023900931B68F3
:102B5000D20B4B439A420CD89B1A3B2B0BD82368C1
:102B600046490B4023602B680B402B60444B1A6096
:102B70001FE7D31AF1E7013EF6B2002ED4D1236845
:102B80003E4A134023602B6813402B603B68042BA4
:102B900007D9BFF34F8F3B4B3B4ADA60BFF34F8FF0
:102BA000FEE780222B68032093432B6001F060F93D
:102BB0002268224B03201A4028231343236001F08C
:102BC00057F9244B009A1B68DB03DB0B13600822C8
:102BD00023689343236097E707222C4D2B6813400B
:102BE000012B02D1002001F0E3FAAB68284A022051
:102BF0001340AB6001F03CF98023AA685B001343EB
:102C0000AB60D6E64A0AFF1F5CF000406866FF1F13
:102C1000000003400180063DBC0003403408000072
:102C2000A40003407102000014100040FFFF3F00A9
:102C30002810004000E100E03075000000FEFEFFBB
:102C4000C4F0004044F000405066FF1F72060000D0
:102C500040F0004064F0004091FCFFFFFF00FFFFE8
:102C60005866FF1FE30C0000E88000005F361E007E
:102C700060361E00C444FF1F28000100FFFFFEFF56
:102C80005466FF1F00ED00E00400FA053CF0004030
:102C9000FFFEFFFF694E336888331B6883F30888A3
:102CA00001F026FA00F018FC654B664A1B68934257
:102CB00007D0002001F01CF90221634A13688B43FE
:102CC0001360FFF703FE614B614C1878C0B201F04E
:102CD0008FF90023A3600233A3605E4B01202360C1
:102CE00001F0C6F80323A36001F0DAF8040001F054
:102CF00047F8050001F0D4F8574B186001F080FA4E
:102D0000564B1968621A531EA14200D2130080224A
:102D1000D203934201D39B029B0A3268D16AC9074E
:102D200000D478E04E491C0C09689BB24C435943CF
:102D30002402090A641803274A49FC3293680A6886
:102D400049489B1A494A4A4E12684A499B18414AC7
:102D500034609A183B400193036892089C46019B9B
:102D60000A6063440360042B03D901323B400A60CC
:102D700003600B684049E418200001F021F93F4F3F
:102D80003D493B68C3183B602000019301F048F9BE
:102D90003B4C2068081838492060884205D9019BBF
:102DA00001333B6001F03CF9216001F049F9354BFA
:102DB0001B78002B0ED000F0E3FF3168324B4A1B2A
:102DC0001B6812189A4233D2591A4919091A2F4806
:102DD00001F02EF82E4C237A002B0FD000F0D0FFFC
:102DE0003168E3684A1B1218934224D9591A4919C9
:102DF000091A284801F01CF800232372264B83F39C
:102E0000088801F0E5F8022001F09AF8002001F0AE
:102E10006FF800F0DDFFDC0199000234641A5900FC
:102E2000641A09214B438033CB40A408E41882E79D
:102E3000FA218900CBE71949DBE7C0466866FF1F26
:102E40000C0AFF1FB641210310000040490AFF1F72
:102E500014100040C4090000100AFF1F340AFF1FAD
:102E6000380AFF1F200AFF1F280AFF1F1C0AFF1F26
:102E70004C66FF1F240AFF1F710200006008FF1F3D
:102E80002C0AFF1F1C09FF1FE408FF1F0010004051
:102E9000740BFF1F3C10004000000020DC05000008
:102EA000A022054B92009B5810B5002B01D09847EB
:102EB00010BD01F0B5F9FBE70000FF1FA122054B93
:102EC00092009B5810B5002B01D0984710BD01F01F
:102ED000A7F9FBE70000FF1FA222054B92009B58B9
:102EE00010B5002B01D0984710BD01F099F9FBE710
:102EF0000000FF1FA322054B92009B5810B5002B2A
:102F000001D0984710BD01F08BF9FBE70000FF1FCF
:102F1000A422054B92009B5810B5002B01D0984776
:102F200010BD01F07DF9FBE70000FF1F70B500F058
:102F300027FF514B1860042001F002F801F0F0F86F
:102F40000400C30702D401F0CBF870BD00224B4B44
:102F50001A604B4B1878013804282CD800F0CAFEB0
:102F600003231B1F2700200000F0FAFE0128ECD0ED
:102F7000444C2378042B71D101F06AF9002806D063
:102F800001F006F9582000F0E3FF0223237003202C
:102F900000F0D6FFD9E7200000F00AFFE6E72000A6
:102FA00000F05EFFE2E7200000F0C2FFDEE7200055
:102FB00001F0BEF8DAE700F063FF0500012808D150
:102FC000314B1B78053B012B03D82000FFF768FF2E
:102FD000CEE72C4B1B78022B01D0052B20D1022DE4
:102FE00028D12A4B9B7BAB431CD12000FFF766FF07
:102FF000254B18780128BBD16405B9D42349252273
:103000004B7B034205D1233A13405A4253412633A6
:103010001A000B7D9342ABD9322001F051F8A7E79B
:10302000022D07D1184B1B78052B11D12000FFF77B
:1030300053FFDDE7012D0BD1012B03D12000FFF75A
:1030400059FF95E7062B03D12000FFF761FF8FE7BB
:10305000200001F0E5F8022D8AD1C9E7032B04D145
:103060000B4B987C01F08CF891E7072B8FD1094B23
:10307000987B01F04DF88AE79C09FF1F9809FF1F14
:103080009009FF1F2309FF1F1C09FF1FA60BFF1F2D
:10309000BC0BFF1FD40BFF1FFA210A4B0A4A490041
:1030A0001A640A4A5A500A4A04395A50094A0831DD
:1030B0009A64094A5A50094A5C315A50084ADA66F9
:1030C0007047C0460000FF1F7D27FF1F7928FF1FA4
:1030D0002D28FF1F8523FF1FED26FF1F011EFF1F49
:1030E000D51DFF1F10B500F0EDFD10BD8023F7B515
:1030F0009C46264B264F01932649274A274D284CAC
:10310000284B02281AD1604638600868264E3040A5
:10311000802636033043086001990978002909D1D7
:103120001660224A2A60224A2260E02219689143EE
:10313000A03A1BE08021C9021160F2E766463E60BA
:103140000F68194E3E408027FF023E430E600199F2
:10315000097800290DD1176001280ED1154A2A607F
:10316000154A2260E02219689143C03A0A431A6066
:10317000F7BD802189021160EEE7E0210F4A02438A
:103180002A600F4A22601A688A43F0E74B0AFF1F41
:10319000E0000340D80003409000034000000340DB
:1031A0005000034040000340FFFFE3FF0280063D64
:1031B000804508220180063D80660822008006982E
:1031C00080550822F8B51E4B80261A68002014008E
:1031D0003440324232D11A681A4F32431A60012207
:1031E0003B68063093433B6000F042FE0122164DDF
:1031F0002B681E432E603B680A2613433B608027E2
:10320000BF00124B1B683B4211D1013EF6B2FF2EAC
:1032100009D17E220E4B1C682B68E40B14409343AB
:1032200023432B6005E0082000F022FEE9E7002E92
:10323000EFD180222B68600893432B60F8BDC04615
:10324000C4F000405CF0004018F0004068F000401E
:1032500060F0004010B500F083FF01215820034AC0
:1032600000F0F6FDFFF7AEFF10BDC046600AFF1F7D
:1032700010B578220021034800F032FE00F0B0FFC4
:10328000002010BD7069FF1F70B5040000F060FFE2
:1032900000230C200B4A010059438D18515C002972
:1032A0000DD0A14208D1012300246B7000F0B0FDC5
:1032B00000F08EFF200070BD01330A2BEBD11224E9
:1032C000F6E7C0467069FF1F70B5040000F040FFCC
:1032D000002319001D000D4A1078002806D0A042D6
:1032E0000CD1557001310C320A29F5D1002B0AD1CD
:1032F00000F076FF00F06CFF002070BD5078461E95
:10330000B0411B18EEE700F083FDF3E77069FF1F83
:10331000F7B504000C20002384460E4D0192674649
:103320005F43E85D7E19A04212D000280BD10A4B02
:103330009C4662461B7808331370019B70707C5565
:103340007160B360FEBD01330A2BE8D10320F9E7B9
:103350000720F7E77069FF1F6C69FF1F8020F8B531
:10336000484BC0051B68C1248360474BFF251A6882
:10337000012313434361454BA4001A68444B402189
:103380001A60444B1A68444B1A60444B1A59AA43BA
:103390001A51C52292009E58AE433143802699505F
:1033A0009F583F49F6010F403E439E509E5880274C
:1033B0003602360A3043985080201A5900020A40DB
:1033C00002431A5104341A59364E3F0432408026C3
:1033D0003A431A511A5936061202120A32431A5146
:1033E00008341A5980260A4002431A51C322920017
:1033F0009F58B446AF4337439F509F58294E0F40C4
:1034000007439F509F583740802636043743802615
:103410009F509F5836063F023F0A37439F50C022B5
:103420001F59AF433A431A511A591202120A16434E
:10343000C6221E5192009C58AC4365462C439C50BA
:103440009C5800250C4020439850C72080001A58F3
:10345000154C1140C02212020A431A50134B1B781C
:10346000DB08AB4201DC0020F8BD2378002B06D03E
:10347000A368002B00D0984701350C34EEE71220EA
:10348000F2E7C0465C45FF1F5845FF1FB0F0004003
:103490006869FF1FB4F000406469FF1F00E100E0AD
:1034A000FF00FFFFFFFF00FF7069FF1F6C69FF1F38
:1034B000030010B51F2809D8072200201340072455
:1034C00004490A78A24313430B7010BD0023062061
:1034D000F5E7C0466C69FF1F034A044913680020E2
:1034E0000B4013607047C0461CF00040FFFFC1FF57
:1034F000054B06491B780A6805485B0702401B0B11
:10350000134300200B6070476C69FF1F1CF00040E4
:10351000FFFFC1FF70B50C25FFF7EAFF0A4B1C78CF
:103520000A4BE4086543ED18002C01D1200070BD62
:103530002B78002B06D06B68002B00D09847013CFD
:103540000C3DF1E71220F2E76C69FF1F6469FF1F71
:1035500007B50422074801A900F034F9019B0133A3
:1035600005D18023044ADB0411680B43136000205B
:103570000EBDC0461C18001114F00040F0B5050047
:103580002026184B87B00493049B002B03D11124F1
:10359000200007B0F0BD002102220B000191009134
:1035A000052000F025FC02230F490A681A42FCD1CD
:1035B0000596059C631E0593002CFAD10B4A1368EF
:1035C000002BFCDA0F276F440121380000F008FDC2
:1035D0003B782B42DCD0052000F04AFC049B013BE9
:1035E0000493D1E7FFFFFF0790C8004000C80040E8
:1035F00007B500F0ADFD80220821D205936A019144
:10360000002B01D10739916202210C4A1160019906
:10361000481E01900029FAD1033111600531019152
:103620000199481E01900029FAD11160002B02D1A6
:103630008022D205936200F0CBFD07BD00C00040A0
:10364000F0B52D4C89B02378002B4FD1FEF75AF9F5
:1036500002232A4F03903A681A42FCD12023069392
:10366000069B5A1E0692002BFAD1254E3368002B7A
:10367000FCDA0120FFF782FF011E02D0112009B001
:10368000F0BD030003220190009005AD9F2000F0E3
:10369000AFFB0321280000F0A3FC02233A681A4282
:1036A000FCD120230793079B5A1E0792002BFAD1C7
:1036B0003368002BFCDA0120FFF760FF0028DDD122
:1036C0000398FEF733F9AA786B7811041B020B43B9
:1036D00029780B4363601300113B0A49052B07D877
:1036E00001239340A3600B60012323700020C6E7F1
:1036F00080231B03F6E7C0464445FF1F90C80040E7
:1037000000C800409808FF1F1E4B30B55A68187853
:103710001D4B85B0D31859424B4101210093002322
:1037200000F036FC194B1A4A02259A6300221A65EA
:1037300010325A658022C4219D65164B1648D2026C
:10374000DA6789004258154B80241A4080231B04F5
:1037500013434350642341200393E40500F078F9B8
:10376000402000F075F96562039D6B1E0393002DE8
:10377000FAD103236362FFF73BFFA562FFF760FF07
:1037800005B030BD5045FF1F95FFFEF700C8004053
:10379000050001FF04E100E000E100E0FFFF00FFA1
:1037A00010B5064B18705960FFF7AEFF00211320CB
:1037B000034AFFF7ADFD002010BDC0465045FF1F76
:1037C0000937FF1FF0B5040085B003920291FEF7A0
:1037D00099F8882263035B0B52051A438023DB05AB
:1037E0009D6A8023274F0092BA68002601901B0330
:1037F0009A420CD9F82326001B041E401C4206D016
:103800008022214B52025E6219680A431A60002D21
:103810000BD100F09DFC02221C4B1A608023DB05BB
:103820005A62013A9A6200F0D3FC0023039A934251
:1038300020D1002D0AD100F08BFC144B03221D6017
:103840008023DB055A629D6200F0C2FC8023BA68C7
:103850001B039A4208D9002E06D000220A4B0C49BD
:103860005A621A680A401A600198FEF75FF8002051
:1038700005B0F0BD009A0299D2181278CA540133EB
:10388000D4E7C0464445FF1F00C8004000C00040C8
:10389000FFFFFEFFF0B587B0029103920400FEF730
:1038A00031F8019000F054FC802302250122234EC0
:1038B000DB0535605D629A6200F08AFC204F3B6850
:1038C0002B42FCD120230493049B5A1E0492002B0C
:1038D000FAD11C4D2B68002BFCDA0120FFF74EFEBD
:1038E000002802D0112007B0F0BD2000039A0299F1
:1038F00000F066FC022304003A681A42FCD120233F
:103900000593059B5A1E0592002BFAD12B68002BBC
:10391000FCDA0120FFF732FE051EE3D100F018FCAF
:1039200080230322DB0535605A629D6200F050FC63
:103930000198FDF7FBFFE0B2D5E7C04600C00040AC
:1039400090C8004000C80040F0B5802687B0040051
:10395000FDF7D8FFF605B36A02250393029000F045
:10396000F7FB0123244F3D607562B36200F030FC29
:10397000224E33682B42FCD120230493049B5A1E11
:103980000492002BFAD11E4D2B68002BFCDA01208B
:10399000FFF7F4FD002802D0112007B0F0BD200091
:1039A00000F036FB0223019032681A42FCD120233A
:1039B0000593059B5A1E0592002BFAD12B68002B0C
:1039C000FCDA0320FFF7DAFD041EE5D100F0C0FBAE
:1039D00080230322DB053C605A629C6200F0F8FB06
:1039E000039B002B01D1FFF703FE0298FDF79EFF1A
:1039F0006B461879D1E7C04600C0004090C800402F
:103A000000C8004007B5000201910422000A01A984
:103A1000FFF740FF0EBD000073B5050005240B4AFB
:103A2000A3005B429B1819686B46DE1D300000F056
:103A30002FFB022804D133782B55013CEFD276BD01
:103A4000052CFCD00128FAD10230F8E71409001146
:103A50001F2807D8012380228340D20591680B4399
:103A6000936070473F2808D8012380222038834084
:103A7000D20551690B435361F3E75F28F1D8012365
:103A8000802240388340D205116A0B431362E8E775
:103A90001F2807D8012280218240C9058B689343E3
:103AA0008B6070473F2808D801228021203882404F
:103AB000C9054B6993434B61F3E75F28F1D80122B5
:103AC000802140388240C9050B6A93430B62E8E7C6
:103AD0001F2810D880230200DB05153A1968012A37
:103AE00006D820229143196019680A431A6070476A
:103AF00001228240F6E73F2811D880230200DB052F
:103B0000353AD968032A06D810229143D960D9687A
:103B10000A43DA60EBE7012220388240F5E75F28AC
:103B2000E5D842238022181A413B8340D205516ACE
:103B300099435162516A0B435362D8E710B50400B0
:103B4000012813D1A022184992050B685B015B097B
:103B500013430B60154B164A19681140154A0A4366
:103B60001A60402219680A431A6010BD0028FCD16F
:103B700001000A2000F0ECF821000B2000F0E8F82A
:103B8000C0220A4B920019680A4340211A601A6841
:103B90008A431A60B022044912060B685B015B0974
:103BA00013430B60E1E7C04614F000401CF00040F6
:103BB0007F00FEFF80FD010072B6074A13680133E3
:103BC00013600422054B1A600023054A136080220B
:103BD000D2055360FEE7C0467808FF1FC0F00040E2
:103BE000C4F00040044B054A1A60054B1A600022DD
:103BF000044B1A607047C046140AFF1F841E000061
:103C0000380AFF1FC4F000400023034A1360034A30
:103C10001360034A1360704754F0004040F10040C5
:103C200044F10040002310B5184C8AB00093019372
:103C30002378012B27D06946012000F0E9FA0028FB
:103C400017D1009B12490293019B06AA0393114BC3
:103C500002A81B680493104B1B68059300F098F8AA
:103C600010220E4906A800F09BF9002804D1FF237A
:103C7000237000200AB010BD0123094A074902A899
:103C8000237000F085F80120F4E7C0466C66FF1F42
:103C900010290011082900110C29001120290011F8
:103CA0007066FF1F13B501246946012000F0B0FAC9
:103CB000034B00940193FFF7B5FF200016BDC046EB
:103CC000BB0B000010B5FFF79FFFFFF7EBFF0028CD
:103CD00002D0024B984710BDFEE7C046E1A20000AB
:103CE00002B4714649084900095649008E4402BC95
:103CF0007047C04602B4714649084900095C490052
:103D00008E4402BC7047C04603B471464908400067
:103D10004900095A49008E4403BC70470000000066
:103D200001B40248844601BC604700BF0D52010047
:103D300001B40248844601BC604700BF85120100FF
:103D400001B40248844601BC604700BFBD5C01006D
:103D500001B40248844601BC604700BFF99E0011CF
:103D600001B40248844601BC604700BF0134010031
:103D700001B40248844601BC604700BF85C1000011
:103D800001B40248844601BC604700BFC95C010021
:103D900001B40248844601BC604700BFDD3F00001B
:103DA00001B40248844601BC604700BFE90B010032
:103DB00001B40248844601BC604700BF09340100D9
:103DC00001B40248844601BC604700BF894400003A
:103DD00001B40248844601BC604700BF855201001F
:103DE00001B40248844601BC604700BFE9F6000008
:103DF00001B40248844601BC604700BF496D010020
:103E000001B40248844601BC604700BFD9B000003D
:103E100001B40248844601BC604700BF21A90000EC
:103E200001B40248844601BC604700BFE9D40000E9
:103E300001B40248844601BC604700BF2D6C0100FC
:103E400001B40248844601BC604700BF116E000007
:103E500001B40248844601BC604700BF016701000D
:103E600001B40248844601BC604700BF053401002C
:103E700001B40248844601BC604700BF01890000CC
:103E800001B40248844601BC604700BFDD0C01005C
:103E900001B40248844601BC604700BFC11501005F
:103EA00001B40248844601BC604700BF156B0100A5
:103EB00001B40248844601BC604700BFE927000006
:103EC00001B40248844601BC604700BF6D0B01008D
:103ED00001B40248844601BC604700BF8D820000E7
:103EE00001B40248844601BC604700BFB70E000021
:103EF00001B40248844601BC604700BF016C010068
:103F000001B40248844601BC604700BF71B00000A4
:103F100001B40248844601BC604700BF19FA0000A2
:103F200001B40248844601BC604700BFA1AF000055
:103F300001B40248844601BC604700BFF53501006A
:103F400001B40248844601BC604700BF1907010064
:103F500001B40248844601BC604700BF79120100E9
:103F600001B40248844601BC604700BFE51201006D
:103F700001B40248844601BC604700BF8B52010077
:103F800001B40248844601BC604700BF8D110100A6
:103F900001B40248844601BC604700BFC56D010002
:103FA00001B40248844601BC604700BFCD4C01000B
:103FB00001B40248844601BC604700BF8937010054
:103FC00001B40248844601BC604700BF090E0000EE
:103FD00001B40248844601BC604700BF79970000E5
:103FE00001B40248844601BC604700BF3D71010036
:103FF00001B40248844601BC604700BF8914010037
:1040000001B40248844601BC604700BFF9A6000025
:1040100001B40248844601BC604700BFA96F01009B
:1040200001B40248844601BC604700BF090E00008D
:1040300001B40248844601BC604700BF75F8000027
:1040400001B40248844601BC604700BFD54401006A
:1040500001B40248844601BC604700BFE94C01003E
:1040600001B40248844601BC604700BFF9ED00007E
:1040700001B40248844601BC604700BF21440000EF
:1040800001B40248844601BC604700BF51B800003B
:1040900001B40248844601BC604700BF8D3800115E
:1040A00001B40248844601BC604700BFE5B200117C
:1040B00001B40248844601BC604700BF5976010044
:1040C00001B40248844601BC604700BF613701006B
:1040D00001B40248844601BC604700BFA9D8000073
:1040E00001B40248844601BC604700BFDD0A0100FC
:1040F00001B40248844601BC604700BFC9A9000062
:1041000001B40248844601BC604700BFB3520100BD
:1041100001B40248844601BC604700BFC1F70000FB
:1041200001B40248844601BC604700BFBD0B0100DA
:1041300001B40248844601BC604700BFF935010064
:1041400001B40248844601BC604700BF6911010008
:1041500001B40248844601BC604700BF75A9000055
:1041600001B40248844601BC604700BFED6801000D
:1041700001B40248844601BC604700BFED6B0100FA
:1041800001B40248844601BC604700BF4DF90000FD
:1041900001B40248844601BC604700BF6DF60000D0
:1041A00001B40248844601BC604700BF9D6A00001C
:1041B00001B40248844601BC604700BFEDA5000081
:1041C00001B40248844601BC604700BF95730100FA
:1041D00001B40248844601BC604700BF9DA90000AD
:1041E00001B40248844601BC604700BFADAE000088
:1041F00001B40248844601BC604700BF53B90000C7
:1042000001B40248844601BC604700BFC16601009A
:1042100001B40248844601BC604700BFE1AC000025
:1042200001B40248844601BC604700BFE9170100A1
:1042300001B40248844601BC604700BFF90D01008B
:1042400001B40248844601BC604700BFC1A500001C
:1042500001B40248844601BC604700BF01D700009A
:1042600001B40248844601BC604700BFCD0C010088
:10427000020000001ABC001101000000E8B90011A2
:104280000200000016BC001101000000B042FF1F38
:1042900002000000F0B9001101000000B463FF1F2C
:1042A0000200000014BC0011030000002863FF1F7F
:1042B00012000000020000001ABC00110100000002
:1042C00030BA00110200000016BC0011010000000D
:1042D0002DBA0011020000003ABA001103000000DC
:1042E0006363FF1F0200000014BC00110300000004
:1042F0007863FF1F0200000016BC001101000000DF
:104300002CBA00110200000038BA001103000000AE
:104310003963FF1F0200000014BC001103000000FD
:104320005A63FF1F020000001ABC001101000000C8
:1043300074BA00110200000016BC00110100000058
:10434000F943FF1F0200000086BA001101000000BF
:104350006BBA00110200000016BC00110100000041
:10436000F843FF1F0200000084BA001101000000A2
:104370008063FF1F0200000016BC00110100000056
:10438000F743FF1F0200000082BA00110100000085
:104390005BBA00110200000016BC00110100000011
:1043A000F643FF1F0200000080BA00110100000068
:1043B00056BA00110200000016BC001101000000F6
:1043C000F543FF1F020000007EBA0011010000004B
:1043D00051BA00110200000016BC001101000000DB
:1043E000F443FF1F020000007CBA0011010000002E
:1043F0004CBA00110202020202020000BD4B001181
:10440000814B0011C8BA0011900118001800FFFF7D
:104410000701020304050602010600000000000077
:10442000000000000000000000000000000000008C
:104430000000000000000300020000001ABC001190
:104440000100000048BB00110200000016BC001172
:1044500001000000A844FF1F0200000052BB001131
:1044600001000000AE63FF1F0200000014BC001139
:10447000030000001C66FF1F0200000016BC0011B4
:1044800001000000A844FF1F0200000050BB001103
:1044900001000000B063FF1F0200000014BC001107
:1044A000030000001466FF1F12000000000100005E
:1044B00000000111FFFF00005048593600000000C5
:1044C0000000000001000000D9BA00110B00050037
:1044D000F7000000B4000028002800283075A00074
:1044E000A000A000A00000080008E001F0001000FB
:1044F000100010001000100010005000500050007C
:1045000010001000D0070000000000000F000100A4
:104510000500307507001000010081FF0000000059
:10452000FF000000E1700011E96E0011796C0011CC
:10453000FFFF0100FF000000FD9A001179980011B3
:10454000919700110000000000000000000008002A
:10455000040000003B0001085902E0018821280006
:10456000FF000000020000001ABC00110100000062
:10457000E0BC00110200000016BC001101000000A8
:10458000E145FF1F0200000012BC00110100000005
:10459000286AFF1F0200000016BC00110100000085
:1045A000E045FF1F0200000010BC001101000000E8
:1045B000DE45FF1F0200000016BC001101000000D4
:1045C000DC45FF1F020000000EBC001101000000CE
:1045D000D445FF1F180018000000900102000003DE
:1045E00002020000020000001ABC001101000000DD
:1045F000F4BC00110200000016BC00110100000014
:104600002446FF1F020000000CBC00110000000047
:10461000000000000200000014BC001103000000B4
:06462000486AFF1F20FFA5
:040000051FFF184180
:00000001FF
